:10000000008000106D010000E5010000EB01000020
:10001000F1010000F7010000FD010000DE74FFEFB8
:1000200000000000000000000000000003020000CB
:1000300009020000000000000F020000150200008D
:100040001B0200001B0200001B0200001B0200003C
:100050001B020000994F00001B0200001B02000061
:100060001B0200001B0200001B0200001B0200001C
:100070001B0200001B0200001B0200001B0200000C
:100080001B020000B94D00001B0200001B02000013
:100090001B0200001B0200001B0200001B020000EC
:1000A000555C0000354200001B0200001B020000EE
:1000B0001B020000DD5A00001B0200001B020000B2
:1000C0001B0200001B0200001B020000B0840000A5
:1000D0000000001028040000B084000000C00720C9
:1000E00000000000280400105043000000C007205A
:1000F0000000000080B489B000AFF860B9607A6099
:10010000BB68FB61FB68BB6100237B610AE0BA69E5
:10011000131DBB61FB69191DF96112681A607B69C7
:1001200004337B617A697B689A42F0D300BF24373D
:10013000BD4680BC704780B485B000AF7860396040
:100140007B68FB600023BB6007E0FB681A1DFA6058
:1001500000221A60BB680433BB60BA683B689A42ED
:10016000F3D300BF1437BD4680BC704780B584B060
:1001700000AF194BFB6013E0FB681A1DFA601B68A7
:10018000BB60FB681A1DFA601B687B60FB681A1D68
:10019000FA601B683B603A687968B868FFF7AAFFA5
:1001A000FB680E4A9342E7D30DE0FB681A1DFA6024
:1001B0001B687B60FB681A1DFA601B683B6039682E
:1001C0007868FFF7B8FFFB68054A9342EDD305F066
:1001D000BBFA07F0FDF9FEE7CC000000E4000000E8
:1001E000F400000080B400AFFEE780B400AFFEE78B
:1001F00080B400AFFEE780B400AFFEE780B400AF8C
:10020000FEE780B400AFFEE780B400AFFEE780B445
:1002100000AFFEE780B400AFFEE780B400AFFEE7BA
:10022000FFFFFFFFFFFFFFFFFFFFFFFFFFFFFFFFDE
:10023000FFFFFFFFFFFFFFFFFFFFFFFFFFFFFFFFCE
:10024000FFFFFFFFFFFFFFFFFFFFFFFFFFFFFFFFBE
:10025000FFFFFFFFFFFFFFFFFFFFFFFFFFFFFFFFAE
:10026000FFFFFFFFFFFFFFFFFFFFFFFFFFFFFFFF9E
:10027000FFFFFFFFFFFFFFFFFFFFFFFFFFFFFFFF8E
:10028000FFFFFFFFFFFFFFFFFFFFFFFFFFFFFFFF7E
:10029000FFFFFFFFFFFFFFFFFFFFFFFFFFFFFFFF6E
:1002A000FFFFFFFFFFFFFFFFFFFFFFFFFFFFFFFF5E
:1002B000FFFFFFFFFFFFFFFFFFFFFFFFFFFFFFFF4E
:1002C000FFFFFFFFFFFFFFFFFFFFFFFFFFFFFFFF3E
:1002D000FFFFFFFFFFFFFFFFFFFFFFFFFFFFFFFF2E
:1002E000FFFFFFFFFFFFFFFFFFFFFFFFFFFFFFFF1E
:1002F000FFFFFFFFFFFFFFFFFFFFFFFFFFFFFFFF0E
:1003000080B582B000AF1A4B00221A70194B002240
:100310001A70194B00221A70184B00221A70184BD1
:100320001B881946174805F07FFB174B00221A60FF
:10033000164B00221A60164B00221A7000237B60B5
:100340000CE014497A6813465B001344DB000B444D
:10035000163300221A707B6801337B607B68632B45
:10036000EFDD012001F028FD00BF0837BD4680BD4C
:1003700036060010340600102D0400103C0D00104D
:10038000681F0010044700103004001034040010EF
:100390003804001040150010F0B5ADF66C7D06AFC6
:1003A000CE4B1B88002B0BD0CD4BDB79012B07D11B
:1003B00000F012FCC94B1B881946CA4805F034FBF3
:1003C00007F2337300221A7007F23273FE221A709A
:1003D00007F23173FE221A7007F5E66307221A70DE
:1003E0000023A7F8463F07F22E7300221A8007F574
:1003F000E56300221A6007F22E7407F1240207F564
:10040000E56107F2337007F5E463039307F5E663EC
:10041000029307F23273019307F23173009323467C
:1004200001F0F8FD0346A7F8463F07F5E5631B68B2
:100430004FF6FF7293420DD107F232731B78FF2BF8
:1004400008D107F231731B78FF2B03D107F2337306
:1004500000221A7007F233731B78002B18D107F2B1
:10046000317407F22E7207F1240107F5E56007F5F4
:10047000E463029307F5E663019307F23273009396
:10048000234601F039FB03461A4607F233731A700C
:10049000B7F8463F012B10D0934B1B78012B04D0AB
:1004A00003F03CFD0346012B07D1B7F8463F184641
:1004B00000F044FC8C4B00221A70002387F84F3F59
:1004C0000023C7F8403F07F1220300221A80874B20
:1004D0001B78012B0CD0022B18D0002B3ED107F239
:1004E00033731B78032B34D1012387F84F3F30E05F
:1004F00007F233731B78032B04D007F233731B7896
:10050000022B28D1012387F84F3F24E007F23373F1
:100510001B78032B03D1012387F84F3F1DE007F21F
:1005200033731B78022B04D007F233731B78012B33
:1005300013D107F5E5631B6807F12202114618463F
:1005400002F0E0FC0346012B07D1012387F84F3F5F
:1005500003E000BF02E000BF00E000BF97F84F3F9C
:10056000012B68D1B7F8463F013B032B66D801A2A7
:1005700052F823F03D060000850500003D0600000E
:100580008505000007F5E5631B681E4607F22E731C
:100590001B889C4607F231731B789E4607F2327324
:1005A0001B781A4607F5E6631B781D4607F12404FD
:1005B00007F5E46102AB03C983E8030001950092EB
:1005C000734662462146304602F0F0FC0346012B9A
:1005D00033D107F5E5631B689C4607F22E731B8831
:1005E0009E4607F231731B781D4607F232731B7863
:1005F0001E4607F5E6631B787B6007F1240207F2CD
:100600003C7407F5E46103AB03C983E803007B682E
:1006100002930196009573466146204600F0E4FB84
:10062000C7F8400FD7F8401F07F23C730122184665
:1006300004F07CFD01E000BF00E000BF0023C7F82C
:100640003C3F07F11C0300221A6007F11C0207F26D
:100650003C731146184600F06FFDC7F83C0FD7F801
:100660003C3F0233132B00F2C28101A252F823F067
:10067000E5080000D7080000EF090000C1060000EF
:100680000B0700001D07000091070000F5070000A0
:100690008B080000AF080000EF090000F30800001D
:1006A000130900003D080000B70800003B070000E8
:1006B000590700007507000061090000F1060000FD
:1006C00007F23C73184600F0D7FE0346002B40F0BB
:1006D0007B81012000F008FB76E100BF681F00105D
:1006E00000470010044700102D0400103C0D0010BE
:1006F00007F23C73184600F0DEFE0346002B40F084
:100700006581162000F0F0FA60E1022000F0ECFABA
:1007100007F23C73184600F009FF68E1B7F8463F5E
:10072000022B40F05581032000F0DEFA07F23C7303
:100730000021184601F034F84AE1B7F8463F022B91
:1007400040F04881102000F0CFFA07F23C730121FD
:10075000184601F025F83DE107F23C7300211846E8
:1007600000F002FF0346002B40F03681112000F01C
:10077000BBFA31E107F23C730121184600F0F4FEA8
:100780000346002B40F02A81122000F0ADFA25E14B
:1007900007F23C731B79A52B11D107F23C735B79EF
:1007A000692B0CD107F23C739B795A2B07D105209A
:1007B00000F09AFA002004F04BF8FFF7A1FD07F2D1
:1007C0003C731B79A52B40F00B8107F23C735B79DE
:1007D000692B40F0058107F23C739B795B2B40F05D
:1007E000FF80052000F080FA012004F031F8FFF7C7
:1007F00087FDF5E007F23C73DB7B184602F05CF9FD
:100800000346012B40F0EE80072000F06DFA07F25E
:100810003C730433184602F097F907F23C731B7BD4
:10082000184602F06BF907F23C735A7B07F23C73EF
:100830009B7B1946104602F071F9D3E007F23C7336
:10084000DB7B184602F038F90346012B40F0CC80E0
:100850000E2000F049FA07F23C730433184602F008
:1008600073F907F23C731B7B184602F047F907F255
:100870003C735A7B07F23C739B7B1946104602F08F
:100880004DF95F4B01221A70AEE007F23C731B7901
:10089000092B02D00D2B06D0A9E0B7F8463F184629
:1008A00000F04CFA02E000F001FA00BF9FE0554B67
:1008B00001221A709BE007F23C731B79022B00F2B5
:1008C000958007F23C731A794F4B1A700F2000F095
:1008D0000BFA00BF8AE04D4B1B780133DAB24B4B69
:1008E0001A7084E04A4B1B780133DAB2484B1A7015
:1008F0007DE007F23C731B79012B03D1454B0122AC
:100900001A7002E0434B00221A700B2000F0ECF941
:100910006DE007F23C731B799BB21B029AB207F29F
:100920003C735B799BB213449AB23B4B1A803A4BAF
:100930001B88002B06D0384B1B88632B02D8364B04
:1009400064221A80344B1B8841F28832934203D9C7
:10095000314B41F288321A800C2000F0C5F946E094
:1009600007F23C735A7A07F234731A7007F23C7339
:100970001A7A07F234735A7007F23C73DA7907F285
:1009800034739A7007F234730122DA7007F23C7301
:100990009A7907F234731A7107F23C735A7907F2A5
:1009A00034735A7107F23C731B799BB203F5FA63F7
:1009B0009AB207F23473DA8007F23473184604F0FF
:1009C00071FA00F039F912E000BF10E000BF0EE04C
:1009D00000BF0CE000BF0AE000BF08E000BF06E077
:1009E00000BF04E000BF02E000BF00E000BFB7F8B6
:1009F000463F022B40F0A4800023C7F8483F9AE00E
:100A00002D040010350600103C0D001034060010B7
:100A1000360600103D0D0010681F00106D49D7F814
:100A2000482F13465B001344DB000B4416331B783E
:100A3000012B7BD16749D7F8482F13465B0013443D
:100A4000DB000B4414331B78012B6FD16149D7F8BD
:100A5000482F13465B001344DB000B4406331D781C
:100A60005C49D7F8482F13465B001344DB000B4466
:100A70001E685849D7F8482F13465B001344DB0023
:100A80000B44043393F800C05249D7F8482F13465B
:100A90005B001344DB000B44053393F800E0D7F808
:100AA000482F13465B001344DB000833494A99186A
:100AB0004848D7F8482F13465B001344DB00034433
:100AC00007331B7898B2434CD7F8482F13465B0086
:100AD0001344DB00234415331B78029301900091EB
:100AE000734662463146284600F080FF3949D7F800
:100AF000482F13465B001344DB000B441033188867
:100B00003449D7F8482F13465B001344DB000B44ED
:100B1000123302461A802F49D7F8482F13465B003C
:100B20001344DB000B44143300221A70D7F8483FFB
:100B30000133C7F8483FD7F8483F632B7FF76EAFC4
:100B400007F1100407F1140207F1240107F108006E
:100B500007F5E463029307F11803019307F10C030F
:100B60000093234602F00CFB0346012B2DD107F125
:100B700008031B687B6007F114031A683A6007F1E9
:100B800010031B6807F10C02126807F118010C68CA
:100B900007F1240C07F23C7607F5E46103AD03C9C5
:100BA00085E803000294019200933B6862467968ED
:100BB000304600F019F9C7F8400FD7F8401F07F288
:100BC0003C730122184604F0B1FA00BF07F65477CF
:100BD000BD46F0BD4015001080B588B000AF124B87
:100BE0001A78124B9A72124B1A78104BDA72114B18
:100BF0001A780E4B1A730D4800F0CAF803461A46CD
:100C00000A4B5A733B461A460E21084800F0F4F985
:100C1000F861F9693B460122184604F087FA00BFE3
:100C20002037BD4680BD00BF340600100000001014
:100C3000360600102C04001080B58AB000AF07F112
:100C40001C03184604F05CF97B8CDBB23033DAB25B
:100C5000154B1A7197F82120134B5A7197F82020E1
:100C6000114B9A71BA7F104BDA717A7F0E4B1A7260
:100C70003A7F0D4B5A720C4800F08AF803461A4628
:100C8000094B9A723B1D1A460B21074800F0B4F934
:100C90007862796A3B1D0122184604F047FA00BFCA
:100CA0002837BD4680BD00BF2C00001080B588B03D
:100CB00000AF0C4800F06CF803461A46094B9A72D4
:100CC0003B1D1A460B21074800F096F9F861F969B7
:100CD0003B1D0122184604F029FA00BF2037BD460B
:100CE00080BD00BF2000001080B586B000AF034675
:100CF000FB71104B1B78012B18D10F4AFB79137134
:100D00000D4800F045F803461A460B4B5A7107F19F
:100D100008031A460621084800F06EF978617969DF
:100D200007F108030122184604F000FA00BF183743
:100D3000BD4680BD3D0D00101000001080B588B08C
:100D400000AF78607B68DAB2104B1A7101F0CCFE0C
:100D500003461A460D4B5A710C4800F019F8034629
:100D60001A460A4B9A7107F10C031A4607210748E5
:100D700000F042F9F861F96907F10C030122184605
:100D800004F0D4F900BF2037BD4680BD1800001024
:100D900080B487B000AF78607B6801331B781B029A
:100DA000FB607B6802331B781A46FB6813440133EF
:100DB000FB600023FB7501233B6109E03B697A6816
:100DC00013441A78FB7D1344FB753B6901333B6187
:100DD0003A69FB689A42F1DDFB7D5B42DBB2184663
:100DE0001C37BD4680BC704790B5ADF6240D00AFF2
:100DF00007F10C04206007F108000160391D0A604A
:100E00003A4613603B461B680133C7F8183807F1B0
:100E10001003C0221A7007F110031322DA7007F1D1
:100E200008031B681B14DAB207F110031A7107F1EB
:100E300008031B681B12DAB207F110035A7107F19D
:100E400008031B68DAB207F110039A71D7F830383B
:100E5000DAB207F11003DA71D7F83438DAB207F1F1
:100E600010031A72D7F83838DAB207F110035A7241
:100E70000023C7F81C3810E0D7F81C383A1D126858
:100E80001A44D7F81C380A33117807F11002D154EC
:100E9000D7F81C380133C7F81C383B46D7F81C2854
:100EA0001B689A42E8DBD7F81C380A3397F84318D6
:100EB00007F11002D154D7F81C380133C7F81C3899
:100EC000D7F81C380A3397F8421807F11002D154AA
:100ED000D7F81C380133C7F81C38D7F81C380A3348
:100EE00097F8411807F11002D154D7F81C38013394
:100EF000C7F81C38D7F81C380A3397F8401807F1A0
:100F00001002D154D7F81C380133C7F81C38D7F871
:100F10001C380A3397F83F1807F11002D154D7F85C
:100F20001C380133C7F81C38D7F81C380A3397F837
:100F30003E1807F11002D154D7F81C380133C7F816
:100F40001C38B7F83C381B0A9BB287F81738B7F83B
:100F50003C3887F81638D7F81C380A3307F11002E6
:100F600097F81718D154D7F81C380133C7F81C3834
:100F7000D7F81C380A3307F1100297F81618D15425
:100F8000D7F81C380133C7F81C38D7F81C380B3396
:100F9000C7F81838D7F81838033BC7F81038D7F80F
:100FA00010381B12DAB207F110035A70D7F8103854
:100FB000DAB207F110039A70D7F81C3803F10A046B
:100FC00007F110031846FFF7E3FE03461A4607F140
:100FD00010031A5507F10C0307F110001A68D7F82F
:100FE000181800F009F8C7F81C08D7F81C3818467C
:100FF00007F62407BD4690BD80B487B000AFF86007
:10100000B9607A60FB681A787B681A7001237B618B
:1010100001233B6139E03B69FA6813441B78C02B1C
:1010200002D0DB2B11D021E07B695A1C7A611A4671
:101030007B681344DB221A707B695A1C7A611A465A
:101040007B681344DC221A701CE07B695A1C7A61AD
:101050001A467B681344DB221A707B695A1C7A613A
:101060001A467B681344DD221A700BE03B69FA686C
:101070001A447B69591C796119467B680B441278C4
:101080001A7000BF3B6901333B61BA683B699A4201
:10109000C1DC7B6918461C37BD4680BC704780B5F3
:1010A00084B000AF786039600023FB603BE03B68B0
:1010B0001A68FB68D31A012B32DDFB687A68134487
:1010C0001B78DB2B13D1FB6801337A6813441B7840
:1010D000DC2B0CD1FB687A681344C0221A70FB68C1
:1010E00001333A687968184600F008FE18E0FB689A
:1010F0007A6813441B78DB2B12D1FB6801337A68C2
:1011000013441B78DD2B0BD1FB687A681344DB2278
:101110001A70FB6801333A687968184600F0EEFDF2
:10112000FB680133FB603B681B68FA689A42BEDBD0
:1011300000BF1037BD4680BD80B58EB000AF78606F
:10114000396000237B630023FB613B6800221A6047
:101150008E4B1B688E4A134401224FF4807118464F
:1011600004F054F8B861894B1A68BB691344874A84
:101170001360BB69002B40F3048100233B6308E04C
:10118000834A3B6B13441B78C02B08D03B6B013365
:101190003B637E4B1B683A6B9A42F1DB00E000BF79
:1011A0003B6B002B02DD386B00F0DAFD01237B6125
:1011B0000123FB620023BB6200237B62744A7B69CC
:1011C00013441B78DB2B0AD17B690133704AD35C53
:1011D000DC2B04D1C023BB620223FB6217E06C4A04
:1011E0007B6913441B78DB2B0AD17B690133684A86
:1011F000D35CDD2B04D1DB23BB620223FB6206E060
:10120000634A7B6913441B78BB620123FB627A69E2
:10121000FB6A13447B615E4A7B6913441B78DB2BBA
:101220000AD17B6901335A4AD35CDC2B04D1C02339
:101230007B620223FB6217E0554A7B6913441B78EB
:10124000DB2B0AD17B690133514AD35CDD2B04D1FE
:10125000DB237B620223FB6206E04D4A7B69134479
:101260001B787B620123FB627A69FB6A13447B6112
:10127000BB6A1B027A6A13443B617B693B630023B0
:101280003B6227E0424A3B6B13441B78C02B02D1E0
:1012900001237B6325E03E4A3B6B13441B78DB2B29
:1012A00002D10223FB620AE0394A3B6B13441B78EC
:1012B000DB2B02D10223FB6201E00123FB623A6BCC
:1012C000FB6A13443B633B6A01333B623A6A3B6906
:1012D0009A4205D02D4B1B683A6B9A42D2DB00E054
:1012E00000BF3B6A002B03D03A6A3B699A420ED09A
:1012F0007B6B012B08D16FF00103FB613B6A033369
:10130000184600F02DFD3CE00023FB6139E03B680E
:101310003A6B1A6000233B630AE03B6B7A68134424
:101320001B493A6B0A4412781A703B6B01333B63DA
:101330003B681B683A6B9A42EFDB3B681B681846B8
:1013400000F00EFD39687868FFF7A9FE3B690333AA
:101350003B613B683A691A607868FFF719FD0346FC
:10136000FB733B69013B7A6813441B78FA7B9A4212
:1013700003D04FF0FF33FB6103E0786800F00AF818
:10138000F861FB6918463837BD4680BD2804001057
:10139000400D001080B485B000AF78600023FB6082
:1013A0007B6803331B78013B152B5FD801A252F8F1
:1013B00023F000BF0D140000191400001F140000DA
:1013C0006D140000251400006D1400002B140000A3
:1013D000371400006D1400003D1400004314000099
:1013E000491400006D140000311400004F14000077
:1013F000551400005B140000611400006D1400001F
:10140000671400006D140000131400000123FB603A
:101410002CE01123FB6029E00223FB6026E003237C
:10142000FB6023E00423FB6020E00523FB601DE05C
:101430000B23FB601AE00623FB6017E00723FB6029
:1014400014E00923FB6011E00A23FB600EE00C238B
:10145000FB600BE00D23FB6008E00E23FB6005E062
:101460000F23FB6002E01023FB6000BFFB681846FF
:101470001437BD4680BC704780B584B000AF78603B
:101480007B6804331B781B04FB607B6805331B7887
:101490001B02FA681343FB607B6806331B781A460D
:1014A000FB681343FB60F86801F07AFB03461846BB
:1014B0001037BD4680BD80B586B000AF786001238F
:1014C000FB757B6804331B781B043B617B68053329
:1014D0001B781B023A6913433B617B6806331B7818
:1014E0001A463B6913433B617B6807331B789BB209
:1014F0001B02FB817B6808331B789AB2FB8913437C
:10150000FB81FB89632B05D87868FFF7B5FF03469D
:10151000FB7506E0FB891946386901F0E1FB0346DB
:10152000FB75FB7D18461837BD4680BD80B584B07D
:1015300000AF78607B6804331B781B04FB607B681A
:1015400005331B781B02FA681343FB607B68063384
:101550001B781A46FB681343FB60F86801F076FCC1
:1015600000BF1037BD4680BD90B488B000AF786032
:101570000B46FB7000237B617B6804331B781B04E4
:101580003B617B6805331B781B023A6913433B615F
:101590007B6806331B781A463B6913433B617B68C3
:1015A0000A331B789BB21B02FB817B680B331B78D1
:1015B0009AB2FB891344FB817B6801331B789BB291
:1015C0001B02BB817B6802331B789AB2BB89134430
:1015D000BB81BB890A3BBB81BB89082B01D9002396
:1015E000D6E00023FB770023BB8310E0BA8B6B4966
:1015F00013465B001344DB000B441B683A699A42B4
:1016000002D10123FB7705E0BB8B0133BB83BB8B8E
:10161000632BEBD9BB8B7B83FB7F012B0DD1FB892C
:10162000002B0AD17A8B5D4913465B001344DB0023
:101630000B44163300221A70A9E0FB7F002B17D150
:101640000023BB830DE0BA8B544913465B0013445F
:10165000DB000B4416331B78002B06D0BB8B013309
:10166000BB83BB8B632BEED900E000BFBB8B7B83BE
:101670007B8B632B00F289807A8B484913465B0091
:101680001344DB000B443A691A607A8B43491346D2
:101690005B001344DB000B441033FA891A807A8B09
:1016A0007B68187A3D4913465B001344DB000B440A
:1016B000043302461A707A8B7B68D879374913460F
:1016C0005B001344DB000B44053302461A707A8B2F
:1016D0007B68587A314913465B001344DB000B44A6
:1016E000063302461A707A8BBB89D8B22B4913464F
:1016F0005B001344DB000B44073302461A700023DF
:10170000BB8315E0BB8B0C337B817B897A681344E8
:101710007A8BB98B1C78214813465B001344DB009D
:1017200003440B44083322461A70BB8B0133BB833E
:10173000BA8BBB899A42E5D37A8B184913465B0072
:101740001344DB000B441233FA891A807A8B134955
:1017500013465B001344DB000B44143300221A7061
:101760007A8B0E4913465B001344DB000B441533A0
:10177000FA781A707A8B094913465B001344DB0030
:101780000B44163301221A7001E001237B617B694F
:1017900018462037BD4690BC704700BF401500106A
:1017A000B0B58CB002AF78600B46FB707B68093334
:1017B0001B783B627B6804331B781B04FB617B68EE
:1017C00005331B781B02FA691343FB617B68063300
:1017D0001B781A46FB691343FB617B6808331B784F
:1017E000BB617B6807331B787B617B6801331B78A7
:1017F0001B023B617B6802331B781A463B6913442A
:101800003B613B69083B3B613B6AD8B2F969BB6904
:10181000DCB27B69DDB27B680A333A6992B201922D
:1018200000932B46224601F077F80346FB60FB68E5
:10183000002B40F0CA80FB78012B40F0A0803B6970
:10184000082B66D8634B1A68F969634813469B00F6
:1018500013449B00034419605E4B1A683B6AD8B27C
:101860005D4913469B0013449B000B44043302461E
:101870001A70584B1A68BB69D8B2574913469B0077
:1018800013449B000B44053302461A70514B1A68EF
:101890007B69D8B2504913469B0013449B000B440C
:1018A000063302461A704B4B1A683B6998B24A4994
:1018B00013469B0013449B000B44083302461A80D6
:1018C00000237B6214E07B6A0A337A681344414A3E
:1018D00012681878404913469B0013449B00CA18AD
:1018E0007B6A13440A3302461A707B6A01337B62B7
:1018F0007A6A3B699A42E6D3364B1B680133354A14
:101900001360344B1B68092B39DD324B00221A60FF
:1019100035E0324B1B78002B31D1314B1B78012B3A
:101920002DD1FB692F4A13603B6ADAB22D4B1A7135
:10193000BB69DAB22B4B5A717B69DAB2294B9A71C7
:101940003B699AB2274B1A8100237B620DE07B6AC8
:101950000A337A6813441978224A7B6A13440A339B
:101960000A461A707B6A01337B627A6A3B699A4243
:10197000EDD31A4B01221A70194B00221A701A4B20
:101980001B78022B21D1F8697B69D9B27B6803F1FE
:101990000A04104B1A6813469B0013449B000E4A1E
:1019A0001344224600F01EFD0346FB72FB7A012B16
:1019B0000BD1084B1B680133064A1360054B1B68AB
:1019C000092B02DD034B00221A60FB6818462837FA
:1019D000BD46B0BD30040010A01E00103804001039
:1019E00066000010380600103C0D001080B586B06F
:1019F00002AF396011461A460346FB710B46BB71B4
:101A000013467B717979BA79F879BB8B0193BB69FD
:101A100000930B46396800F07FFF0346BB60BB684C
:101A2000002B60D197F82030012B5CD1304B1A6825
:101A3000304913469B0013449B000B443A681A60DC
:101A40002B4B1A682B4913469B0013449B000B44F5
:101A50000433FA791A70264B1A68264913469B00FC
:101A600013449B000B440533BA791A70204B1A6853
:101A7000204913469B0013449B000B4406337A799C
:101A80001A701B4B1A681B4913469B0013449B009A
:101A90000B440833BA8B1A800023FB6013E0FB6809
:101AA000BA691344124A12681878124913469B0007
:101AB00013449B00CA18FB6813440A3302461A7089
:101AC000FB680133FB60BB8BFA689A42E7DB084B8B
:101AD0001B680133064A1360054B1B68092B02DDA6
:101AE000034B00221A60BB6818461037BD4680BD04
:101AF00030040010A01E001080B586B000AFF86062
:101B0000B9607A603B60FB6800221A607B68002243
:101B10001A803B68FE221A703B6AFE221A707B6AAA
:101B200000221A7000BF674B1B78002BFBD0664B5E
:101B30001A78BB6ADA71654B1A78BB6A9A71644B82
:101B40001A78BB6A5A71634B1A78BB6A1A71624B76
:101B50001A78BB6ADA70614B1A78BB6A9A70604B6C
:101B60001A88BB6A1A805F4B1A685F4B1B689A42DF
:101B70006DD05C4B1A685D4913469B0013449B0073
:101B80000B441A68FB681A60564B1A68574913468B
:101B90009B0013449B000B4404331A787B6A1A7031
:101BA000504B1A68514913469B0013449B000B4449
:101BB00005331A783B6A1A704A4B1A684B49134628
:101BC0009B0013449B000B4406331A783B681A7041
:101BD000444B1A68454913469B0013449B000B4431
:101BE00008331A887B681A8000237B6112E03D4B22
:101BF0001A687B69B96819443C4813469B00134432
:101C00009B00C2187B6913440A331B780B707B69F5
:101C100001337B617B681B881A467B699342E6DB54
:101C2000304B1B6801332F4A13602E4B1B68092B66
:101C300002DD2C4B00221A60B968F86800F0C6FE7D
:101C40000346012B01D1012338E0032336E0284B62
:101C50001B78012B31D1274B1B78012B2DD1264B23
:101C60001A68FB681A60244B1A797B6A1A70224B37
:101C70005A793B6A1A70204B9A793B681A701E4B4E
:101C80001A897B681A8000237B610BE07B69BA6844
:101C9000134419497A690A440A3212781A707B6926
:101CA00001337B617B681B881A467B699342EDDBBD
:101CB0000F4B00221A70032300E000231846183748
:101CC000BD4680BD450400106E0000106D00001080
:101CD0006C0000104A040010490400104804001071
:101CE000460400103404001030040010A01E001040
:101CF00038040010660000103806001080B489B067
:101D000000AFF860B9607A60FB680133FB61FB6883
:101D1000BB6100237B6110E0FB695A1CFA611A4623
:101D2000BB681A44BB69591CB9611946BB680B44AE
:101D300012781A707B6901337B617B681A68FB68D3
:101D4000D31A013B7A699A42E6DB7B681B685A1E0C
:101D50007B681A6000BF2437BD4680BC7047FFFF18
:101D600080B487B000AF78607B687B6100233B6103
:101D70000F4B1A687B68D31A0D4A13600023FB606F
:101D80000CE07A69531C7B613B69591C3961094934
:101D9000895C084AD154FB680133FB60044B1B6823
:101DA000FA689A42EDDB00BF1C37BD4680BC704725
:101DB00028040010400D001080B584B000AF78609A
:101DC000814800F0F1FD814800F0EEFDFA227B68C9
:101DD00092FBF3F39AB27E4B1A8064227B6892FBEB
:101DE000F3F39AB27B4B1A8008227B6892FBF3F3E1
:101DF0009AB2794B1A8009227B6892FBF3F39AB26C
:101E0000754B5A800A227B6892FBF3F39AB2724BAD
:101E10009A800C227B6892FBF3F39AB26E4BDA80C5
:101E20000F227B6892FBF3F39AB26B4B1A8100236B
:101E3000FB8133E0FA89694913469B001344DB00B8
:101E40000B4400221A70FA89644913469B0013441C
:101E5000DB000B44043300221A60FA895F49134601
:101E60009B001344DB000B44083300221A80FA89DC
:101E70005A4913469B001344DB000B440A330022EB
:101E80001A80FA89554913469B001344DB000B4422
:101E9000143300221A80FB890133FB81FB89632BF9
:101EA000C8D94F4B00221A704D4B00225A704C4B30
:101EB00000229A704A4B0022DA70494B00221A71B4
:101EC000474B00225A71464B00229A71444BFE2226
:101ED000DA71434BFE221A72414BFE225A72404B7A
:101EE00000229A723E4BFE22DA723D4BFE221A739A
:101EF0003B4B00229A733A4B00225A7332227B6882
:101F000092FBF3F39AB2374B1A8040F2EE227B68D1
:101F100092FBF3F39AB2344B1A8032227B6892FB25
:101F2000F3F39AB2314B1A8040F2EE227B6892FBB7
:101F3000F3F39AB22E4B1A80C8227B6892FBF3F31C
:101F40009AB22C4B1A804FF4FA727B6892FBF3F32F
:101F50009AB2294B1A8040F2EE227B6892FBF3F38F
:101F60009AB2234B1A8040F2E2427B6892FBF3F371
:101F70009AB2224B1A8040F2E2427B6892FBF3F362
:101F80009AB21F4B1A8040F21A427B6892FBF3F31D
:101F90009AB21C4B1A80002001F028FF002001F0AB
:101FA00063FF194B00221A70184B01221A70184B4C
:101FB0001B6801221946012002F058FA0346184610
:101FC0001037BD4680BD00BF084700100C47001009
:101FD00044360010781F00105C000010A42600108A
:101FE0007C1F00109E260010623D0010603D001016
:101FF0006C1F0010A02600109C260010583D0010F9
:102000005E3D00105C3D00105A3D0010660000105F
:102010006800001090B58BB004AFF860B9607A60CA
:102020003B600423FB757B6B02933B6B0193FB6A64
:102030000093BB6A3A687968B86800F001FC03460F
:102040001A46FB681A70FB681B78032B1BD1BB6810
:102050001B6807F110021146184600F053FF0346B3
:10206000012B0DD1BB6A1A78A34B1B7B9A420AD075
:10207000BB6A1B78FF2B06D0FB6802221A7002E0B5
:10208000FB6800221A709C4B1B78002B01D1FB7D52
:102090009AE1994B9B78012B40F036810223FB7526
:1020A000BB681B68B3F56E4F42D04FF6D8629342BF
:1020B00000F09080B3F56A4F40F09180FB681B7888
:1020C000012B40F089807B681B78002B40F08480D6
:1020D0007B6801331B78EE2B7ED17B6802331B7843
:1020E000002B79D1BB6A1B78FF2B0CD1824B1A7B5A
:1020F00008230193814B0093FF234FF46E41062088
:1021000000F00AFC68E0BB6A1A787B4B1B7B9A42A2
:1021100062D1794B1A7BFB6A197808230193774BBC
:1021200000930B464FF46E41062000F0F5FB53E0A0
:10213000FB6A1A78704B1B7B9A4249D16F497868C9
:1021400000F04EFB0346FB74FB7C012B1DD0022BE1
:1021500031D0002B42D1002001F048FE002001F0D8
:1021600083FE08230193654B0093FF23FE224FF467
:102170006E41062000F0D0FB5F4B00229A705E4B50
:1021800001229A710323FB7523E0002001F02EFE4B
:10219000002001F069FE584B00225A70564B002275
:1021A0009A70FB6A1B785549184600F073F9524B38
:1021B00001221A710DE0504B1A7B082301934F4BFB
:1021C0000093FF234FF46E41062000F0A5FB00E0D2
:1021D00000BF03E000BF02E000BF00E000BFBB683B
:1021E0001B68B3F56C4F04D0BB681B68B3F56B4F2D
:1021F00002D1FB6800221A70BB6818683B68198816
:10220000BB6A1C78FB6A1B783A6B127801920093C8
:1022100023460A46796801F0BDF8FB681B78002B5D
:1022200040F0D180364B93F80C37012B2ED1344B34
:102230009A68BB681A60324BB3F80A273B681A8069
:102240002F4B5A7BBB6A1A702D4B1A7BFB6A1A7094
:102250003B6BFF221A700023BB820AE0BA8ABB8A5A
:1022600079680B4426490A44127C1A70BB8A0133F0
:10227000BB82234BB3F80A37BA8A9A42EED30020C6
:1022800001F0B4FDFB6803221A709CE01D4B93F82B
:102290000C37012B40F097801A4B9A68BB681A6084
:1022A000184BB3F80A273B681A80164B5A7BBB6A57
:1022B0001A70144B1A7BFB6A1A703B6BFF221A7060
:1022C0000023BB820AE0BA8ABB8A79680B440D49B5
:1022D0000A44127C1A70BB8A0133BB82094BB3F8E3
:1022E0000A37BA8A9A42EED3002001F0BDFDFB689E
:1022F00003221A7067E000BF7C1F00103800001036
:10230000483600108C1F0010314B9B79012B52D1A5
:102310000323FB75BB681B68B3F56E4F33D04FF6D4
:10232000D862934231D0B3F56A4F31D1FB681B7844
:10233000012B2CD17B681B78002B28D17B680133C3
:102340001B78EE2B23D17B6802331B78002B1ED128
:10235000BB6A1B78FF2B1AD11D4B9B7B5A1CD1B239
:102360001B4A91731A461B4B33F812201A4B9A8161
:10237000194B01229A73164B9B7B042B07D9144BE4
:1023800000229A7303E000BF02E000BF00E000BF3C
:10239000114BDB7B012B16D1104800F005FB082305
:1023A00001930F4B0093FF23FE224FF46E41062052
:1023B00000F0B2FA07E0FB6A1B787968184600F073
:1023C00069F80346FB75FB7D18461C37BD4690BD7A
:1023D0007C1F00105C000010004700100C4700102C
:1023E0003800001080B588B002AFF8607A603B60BA
:1023F0000B46FB720023FB75FB68B3F56A4F40D1B7
:10240000FB7AFF2B3DD17B681B78002B39D17B6891
:1024100001331B78EE2B34D17B6802331B78002B01
:102420002FD11A4B1A7B08230193194B0093FF23DA
:102430004FF46E41062000F06FFA3B684FF46E4295
:102440001A603B6806221A71104B1A7B3B685A715E
:102450003B68FF229A713B6808221A810023BB82E5
:102460000AE0BA8ABB8A0A49895C3A6813440A4678
:102470009A72BB8A0133BB82BB8A072BF1D9012335
:10248000FB75FB7D18461837BD4680BD7C1F0010CC
:102490003800001080B586B002AF03463960FB718A
:1024A0000123FB73954B9B79012B02D10323FB7313
:1024B0001EE1924B9B78012B02D10223FB7317E1A3
:1024C0008E4B5B79012B1ED18D4BDB7B012B40F0BA
:1024D0000F818C4800F068FA884BDA7A0823019360
:1024E000894B0093FF234FF46E41062000F014FA4D
:1024F000864B1A88824B1A81814B01229A727F4B3C
:1025000000225A71F4E07D4B5B78002B2FD100F054
:1025100007F90346012B16D1784BDA7A0823019389
:10252000794B0093FF234FF46E41062000F0F4F93D
:10253000764B1A88724B1A81714B01229A726F4B3B
:1025400001225A70D4E0082301936F4B0093FF23BC
:10255000FE224FF46E41062000F0DEF9674B0022A8
:102560009A70664B01229A710323FB73C0E0644B9F
:10257000DB7A012B0CD1664800F016FA5F4BDA7A51
:102580005E4B1A735D4B01229A700223FB73AFE01E
:10259000012001F043FF0346012B35D15C4800F0D8
:1025A00003FA5C4B1B780133DAB25A4B1A70594B61
:1025B0001B78142B08D1514B00229A704F4B0122EB
:1025C0009A710323FB731FE0534B1B6801221946CA
:1025D000012001F04BFF494B9B7B5A1CD1B2474A6B
:1025E00091731A464D4B33F81220454B9A81444B58
:1025F00001229A73414B9B7B042B02D93F4B002253
:102600009A733E4B01225A713C4BDB7AFA799A421B
:102610006DD13D49386800F0E3F80346BB73BB7BDE
:10262000012B1DD0022B4ED0002B61D1002001F0D8
:10263000DDFB002001F018FC08230193324B0093CE
:10264000FF23FE224FF46E41062000F065F92B4B6C
:1026500000229A70294B01229A710323FB7347E0F1
:10266000002001F0C3FB002001F0FEFB00F058F851
:102670000346012B13D1214BDA7A08230193224B15
:102680000093FF234FF46E41062000F045F91F4BE5
:102690001A881B4B1A811A4B01229A7228E00823D0
:1026A0000193194B0093FF23FE224FF46E41062045
:1026B00000F032F9114B00229A70104B01229A71EE
:1026C0000323FB7314E00D4BDA7A082301930E4BBE
:1026D0000093FF234FF46E41062000F01DF90B4BD1
:1026E0001A88074B1A81064B01229A7200E000BF3C
:1026F000FB7B18461037BD4680BD00BF7C1F001015
:10270000004700100C47001038000010443600103D
:10271000084700105A3D0010680000105C000010CF
:1027200080B483B000AF0123FB712C4BDB79FE2B0F
:1027300002D12A4B0122DA70284BDB78002B07D11B
:10274000264BDA79254BDA72244B0122DA703EE00F
:10275000224B1B7AFE2B03D0204B5B7AFE2B02D13F
:102760000023FB7133E01D4BDB7AFE2B03D01B4BA8
:102770009B7A002B07D1194B1A7A184BDA72174B38
:1027800001229A720EE0154BDA7A144B5B7A9A4268
:1027900006D2124BDB7A0133DAB2104BDA7201E067
:1027A0000023FB710D4BDA7A0C4BDB799A420ED188
:1027B0000A4BDA7A094B5B7A9A4206D2074BDB7AEC
:1027C0000133DAB2054BDA7201E00023FB71FB79C9
:1027D00018460C37BD4680BC704700BF7C1F0010F8
:1027E00080B485B000AF786039600823FB731EE0C9
:1027F000FB7B013B7A6813441A78FB7B013B396809
:102800000B441B789A420FD0FB7B013B7A68134440
:102810001A78FB7B013B39680B441B789A4201D242
:10282000012308E0022306E0FB7B013BFB73FB7BFB
:10283000002BDDD1002318461437BD4680BC7047FD
:1028400080B58AB002AFF860B9607A603B60FB681F
:1028500000221A607B6800221A803B68FE221A70F0
:10286000BB6AFE221A70FB6A00221A7007F114027A
:1028700007F110013B6B00931346BA68012001F089
:102880003DFE0346002B3FD13B69FB617B699AB259
:102890007B681A80FB6903F0E053BB61BB699B0E48
:1028A000DAB2FB6A1A70FB6923F07E4323F0FF0360
:1028B000FA681360FB681B681A0AFB681A60FB69F8
:1028C000DAB2BB6A1A703B68FF221A70FB681B6899
:1028D000184600F0D7F80346012B0AD1FB681B68A5
:1028E000DAB23B681A70FB681A680A4B1340FA6840
:1028F0001360B968F86800F069F80346012B01D14C
:10290000012302E0032300E0002318462037BD46E0
:1029100080BD00BF00FF010080B586B002AF396006
:1029200011461A460346FB710B46BB7113467B7179
:10293000BB8B40F2F962934201D9012330E0FB796D
:102940009A063B681B021A44BB791344FB60386843
:1029500000F098F80346012B08D1FB6823F47F436D
:10296000FB607B791B02FA681343FB60BB8B082B6F
:102970000CD97979BA79F879BB8B0193BB6900934B
:102980000B46396801F0B2F9034609E0F968BA8BE1
:10299000002300931346BA69012001F015FF034696
:1029A00018461037BD4680BD80B483B000AF786054
:1029B0007B6800221A807B6800229A707B68002264
:1029C000DA7000BF0C37BD4680BC704780B485B05C
:1029D00000AF786039600023FB737B681B681B0ABB
:1029E0007B737B681B683B737B7BEA2B2AD13B7B29
:1029F000FF2B10D13B681B78002B39D13B6801338A
:102A00001B78EE2B34D13B6802331B78002B2FD17F
:102A10000123FB732CE07B681B6803F47F427B6817
:102A20001A603B681B78002B22D13B6801331B786E
:102A3000EE2B1DD13B6802331B78002B18D10123EC
:102A4000FB7315E00023BB730EE07B681A68BB7B49
:102A50000B4951F823309A4203D10123FB7300BF85
:102A600007E0BB7B0133BB73BB7B032BEDD900E0DD
:102A700000BFFB7B18461437BD4680BC704700BFC3
:102A80004000001080B483B000AF78607B68B3F57D
:102A9000704F01D201230AE07B68B3F5803F05D374
:102AA0007B68B3F5F83F01D2012300E0002318460C
:102AB0000C37BD4680BC704780B485B000AF03467C
:102AC000FB710023FB73FB79012B04D1054AFB79D1
:102AD00013700123FB73FB7B18461437BD4680BC83
:102AE000704700BF7C1F001080B400AF024B1B7BFF
:102AF0001846BD4680BC70477C1F001080B483B070
:102B000000AF0346FB71044AFB79D37100BF0C3759
:102B1000BD4680BC704700BF7C1F001080B483B0EE
:102B200000AF03460A46FB711346BB71054AFB79A9
:102B30001372044ABB79537200BF0C37BD4680BC88
:102B4000704700BF7C1F001080B483B000AF786076
:102B50007B681A78114B1A707B685A780F4B5A7041
:102B60007B689A780D4B9A707B68DA780B4BDA7039
:102B70007B681A79094B1A717B685A79074B5A712D
:102B80007B689A79054B9A717B68DA79034BDA7125
:102B900000BF0C37BD4680BC704700BF3800001036
:102BA00080B584B000AF78600123FB737B6803F4C9
:102BB0007F43B3F56A4F02D14FF46A437B607B6871
:102BC00003F47F43B3F56E4F02D14FF46E437B6045
:102BD0007B68B3F5801F05D13F4B01225A73002358
:102BE000FB7373E007F10A031946786800F08AF96D
:102BF0000346012B23D17B891946384A0B469B009B
:102C00000B44DB001344083300221A807B891946E9
:102C1000324A0B469B000B44DB0013440A3300226C
:102C20001A807B8919462D4A0B469B000B44DB001A
:102C30001344143300221A800023FB7346E0002360
:102C4000BB8140E0BA89254913469B001344DB0051
:102C50000B441B78002B33D1BA89204913469B00C3
:102C60001344DB000B4401221A70BA891B49134636
:102C70009B001344DB000B4404337A681A60BA8962
:102C8000164913469B001344DB000B440833002213
:102C90001A80BA89114913469B001344DB000B4488
:102CA0000A3300221A80BA890C4913469B00134448
:102CB000DB000B44143300221A800023FB7305E071
:102CC000BB890133BB81BB89632BBBD9FB7B184616
:102CD0001037BD4680BD00BF7C1F0010A426001029
:102CE00080B584B000AF78600B467B800123FB7316
:102CF0007B88632B04D87868FFF752FF03469EE079
:102D00007B6803F47F43B3F56A4F01D1FB7B96E008
:102D10007B6803F47F43B3F56E4F01D1FB7B8EE0FC
:102D20007B68B3F5801F01D1FB7B88E007F10A03C4
:102D30001946786800F0E6F80346012B37D17B8905
:102D40001946414A0B469B000B44DB00134400220A
:102D50001A707B8919463C4A0B469B000B44DB00EA
:102D6000134408337A881A807B891946364A0B4601
:102D70009B000B44DB0013440A337A881A807B895A
:102D80001946314A0B469B000B44DB0013441433B5
:102D900000221A807B8919462B4A0B469B000B4464
:102DA000DB00134401221A700023FB7346E000236A
:102DB000BB8140E0BA89244913469B001344DB00E1
:102DC0000B441B78002B33D1BA891F4913469B0053
:102DD0001344DB000B4404337A681A60BA891A4939
:102DE00013469B001344DB000B4408337A881A8097
:102DF000BA89154913469B001344DB000B440A3380
:102E00007A881A80BA89104913469B001344DB0064
:102E10000B44143300221A80BA890B4913469B00D5
:102E20001344DB000B4401221A700023FB7305E0FE
:102E3000BB890133BB81BB89632BBBD9FB7B1846A4
:102E40001037BD4680BD00BFA426001080B485B0F9
:102E500000AF78607B6803F47F43B3F56A4F02D11B
:102E60004FF46A437B607B6803F47F43B3F56E4F96
:102E700002D14FF46E437B607B68B3F5801F03D1B2
:102E80001E4B00225A7333E00023FB812DE0FA89A8
:102E90001B4913469B001344DB000B4404331B689F
:102EA0007A689A421ED1FA89154913469B00134449
:102EB000DB000B4400221A70FA89114913469B006B
:102EC0001344DB000B44043300221A60FA890C49D6
:102ED00013469B001344DB000B44083300221A8086
:102EE00000BF05E0FB890133FB81FB89632BCED951
:102EF00000BF1437BD4680BC704700BF7C1F001068
:102F0000A426001080B485B000AF7860396000233B
:102F1000FB733B684FF6FF721A80224B5B7B012BE1
:102F200002D10123FB7336E07B6803F47F43B3F5E2
:102F30006A4F02D14FF46A437B607B6803F47F439E
:102F4000B3F56E4F02D14FF46E437B600023BB811B
:102F50001EE0BA89144913469B001344DB000B445E
:102F60001B78012B11D1BA890F4913469B001344DA
:102F7000DB000B4404331B687A689A4205D10123B5
:102F8000FB733B68BA891A8005E0BB890133BB81BA
:102F9000BB89632BDDD9FB7B18461437BD4680BC4B
:102FA000704700BF7C1F0010A426001090B587B0AA
:102FB00000AFF860B9607A603B6000237B82002339
:102FC0007B756D4B5B7B012B02D101237B75CDE0C3
:102FD000FB6807F1120211461846FFF793FF0346FC
:102FE000012B40F0C3807B8A1946644A0B469B0044
:102FF0000B44DB00134408331B88002B00F0B48023
:103000007B8A1846FA685D4903469B000344DB004F
:103010000B4404331A607B8A1946FB6AD8B2574ABC
:103020000B469B000B44DB001344103302461A701E
:103030007B8A1946BB6AD8B2504A0B469B000B44A8
:10304000DB001344113302461A707B8A19463B6831
:10305000D8B24A4A0B469B000B44DB0013441233A0
:1030600002461A707B8A19467B6898B2434A0B461F
:103070009B000B44DB001344143302461A800023E8
:10308000FB8213E0FB8ABA6813447A8A1046FA8AF4
:103090001C783A4903469B000344DB000B4413446D
:1030A000163322461A70FB8A0133FB82FB8A072BF8
:1030B000E8D97B8A1946388E304A0B469B000B4470
:1030C000DB001344203302461A807B8A194697F8A6
:1030D00032002A4A0B469B000B44DB001344223388
:1030E00002461A707B8A194697F83300234A0B462A
:1030F0009B000B44DB001344233302461A707B8A87
:10310000194697F834001D4A0B469B000B44DB0020
:103110001344243302461A707B8A194697F8350007
:10312000164A0B469B000B44DB0013442533024632
:103130001A707B8A194697F83600104A0B469B0096
:103140000B44DB001344263302461A707B8A19466F
:1031500097F83700094A0B469B000B44DB001344E9
:10316000273302461A7001E001237B757B7D1846E8
:103170001C37BD4690BD00BF7C1F0010A426001068
:1031800080B489B000AFF860B9607A603B6000231A
:10319000FB750023FB61F1E07D49FA6913469B0052
:1031A0001344DB000B441B78012B40F0E48078498A
:1031B000FA6913469B001344DB000B4408331B8859
:1031C000002B00F0D8807249FA6913469B00134423
:1031D000DB000B440A331B88002B40F0CC806C4989
:1031E000FA6913469B001344DB000B4414331B881D
:1031F000002B00F0C0800123FB756549FA69134676
:103200009B001344DB000B4404331B681A46FB6825
:103210001A605F49FA6913469B001344DB000B44B4
:1032200014331B881A467B681A600023BB6111E0C7
:10323000BB69BA68D1185648FA6913469B00134413
:10324000DB00C218BB69134416331B780B70BB69D3
:103250000133BB61BB69072BEADD4D49FA691346AF
:103260009B001344DB000B4412331B781A463B6867
:103270001A604749FA6913469B001344DB000B446C
:1032800011331B781A46BB6A1A604149FA69134622
:103290009B001344DB000B4410331B781A46FB6A77
:1032A0001A603B49FA6913469B001344DB000B4448
:1032B00020331A883B6B1A803549FA6913469B0004
:1032C0001344DB000B4422331A783B6B9A7030496D
:1032D000FA6913469B001344DB000B4423331A782E
:1032E0003B6BDA702A49FA6913469B001344DB00F2
:1032F0000B4424331A783B6B1A712549FA6913463B
:103300009B001344DB000B4425331A783B6B5A7146
:103310001F49FA6913469B001344DB000B44263314
:103320001A783B6B9A711A49FA6913469B00134449
:10333000DB000B4427331A783B6BDA711449FA69C6
:1033400013469B001344DB000B44083318881049D4
:10335000FA6913469B001344DB000B440A33024610
:103360001A800B49FA6913469B001344DB000B4497
:10337000143300221A80FB690133FB61FB69632B64
:103380007FF70AAFFB7D18462437BD4680BC7047E7
:10339000A426001080B58AB002AFF860B96011466B
:1033A0001A460B46FB8013467B710023FB77974B35
:1033B0001B78022B40F09580944B5B78012B40F0FA
:1033C0009080924B9B78002B41D1914B20221A7018
:1033D0008E4BB3F80A37DAB28D4B5A708B4BB3F879
:1033E0000A371B0A9BB2DAB2894B9A70874B9A7BD9
:1033F000874BDA70864BFF221A71844B9B68DAB2D6
:10340000834B5A71814B9B681B0ADAB2804B9A71CD
:103410007E4B9B681B0CDAB27D4BDA717B4B1A7BBF
:10342000082301937A4B0093FF234FF46C4107204C
:10343000FFF772FA0346FB77764B1A88764B1A82AF
:10344000754B01229A74714B01229A7049E0724BBC
:10345000DB7C012B45D16D4BDB7B9BB21A46D20046
:10346000D31ABB83694BDB7B0133DAB2674BDA7368
:10347000664BDA7B694B1A7000237B830CE0BA8BB6
:103480007B8B1A447B8B013360490A44117C634A6D
:10349000D1547B8B01337B837B8B062BEFD95B4B2A
:1034A0001A7B082301935D4B0093FF234FF46B417C
:1034B0000720FFF731FA0346FB77544BDA7B534B77
:1034C0009B7B9A4203D1002000F090FC09E0514B15
:1034D0001A88514B1A82504B01229A744E4B00228B
:1034E000DA74FB68B3F56C4F5FD1BB681B78202B97
:1034F0005BD1464B1B78002B57D1444B93F80C37CC
:10350000002B52D1BB6807331B781A04BB68063303
:103510001B781B021344BA680532127813443B4AE5
:1035200093603A4B9B6807F1160211461846FFF765
:10353000E9FC0346012B35D1BB6801331B789AB2F5
:10354000BB6802331B789BB21B029BB213449AB236
:103550002E4BA3F80A272D4BB3F80A3740F2F96235
:10356000934203D9002000F041FC1EE0274B0122CA
:103570001A70264B01225A70244A97F82830137388
:10358000224A7B795373BB68DA78204B9A731F4BBE
:103590000022DA73224B1A881F4B9A821E4B01229B
:1035A0009A7502E0194B00229A60184B1B78012B88
:1035B00006D1194BDB7D012B02D1002000F016FC57
:1035C000124B1B78012B51D1104B5B78012B4DD145
:1035D000FB68B3F56B4F49D10C4B1B7B97F8282048
:1035E0009A4243D1094B5B7B7A799A423ED10C4B8C
:1035F0001A88094B9A82BB681B78013B9BB21A461A
:10360000D200D31ABB8301237B8319E04836001014
:10361000500000109E26001000470010701F001080
:10362000623D00107B8BBA681A44BB8B591CB9836E
:1036300019461278994B0B441A747B8B01337B83A8
:103640007B8B072BEED9954BDB7B0133DAB2934BA7
:10365000DA73924BDA7B914B9B7B9A4206D1012025
:1036600000F0C4FB8D4B012283F80C278C4B1B7898
:10367000022B0ED18A4B5B78012B0AD1FB68B3F584
:103680006C4F06D1BB681B78FF2B02D1002000F0E5
:10369000EBFB834B1B78022B0ED1814B5B78012B0C
:1036A0000AD1FB68B3F56C4F06D1BB681B78132BAE
:1036B00002D1002000F0D8FB794B1B78022B40F0A0
:1036C0004381774B5B78012B40F03E81744BDB7874
:1036D000002B43D1734B10221A70714BB3F80A3789
:1036E000DAB2704B5A706E4BB3F80A371B0A9BB2B2
:1036F000DAB26C4B9A706A4B9A7B6A4BDA70694B00
:10370000FF221A71664B9B68DAB2664B5A71644BA2
:103710009B681B0ADAB2634B9A71614B9B681B0C66
:10372000DAB2604BDA715E4B1A7B5D4B597B082332
:1037300001935C4B00930B464FF46C410720FFF75D
:10374000EBF80346FB77584B1A88584B9A83574B34
:1037500001229A77524B0122DA70F5E0534BDB7F5E
:10376000012B32D14F4BFF221A704E4B03225A705D
:103770004C4BFF229A704B4BFF22DA70494BFF22D1
:103780001A71474B9B68DAB2464B5A71444B9B689F
:103790001B0ADAB2434B9A71414B9B681B0CDAB29D
:1037A000404BDA713E4B1A7B3D4B597B082301930A
:1037B0003C4B00930B464FF46C410720FFF7ACF8ED
:1037C0000346FB77002000F04FFBFB68B3F56C4F1E
:1037D00015D1334B1B7B7A799A4210D1BB681B7889
:1037E000112B0CD13248FFF7DFF8324B1A882F4BE0
:1037F0001A832E4B01229A76294B01221A71284BEB
:103800001B79012B68D1294BDB7E012B64D1244B22
:10381000DB7B9BB21A46D200D31ABB83204BDB7BE7
:103820000133DAB21E4BDA731D4BDA7B224B1A706E
:1038300000237B830CE0BA8B7B8B1A447B8B013398
:1038400017490A44117C1C4AD1547B8B01337B837A
:103850007B8B062BEFD9124B1A7B114B597B08231C
:103860000193154B00930B464FF46B410720FFF774
:1038700053F80346FB770A4BDA7B094B9B7B9A4252
:1038800020D10E48FFF790F80D4B1A88074B9A8508
:10389000064B012283F82E201EE000BF48360010A0
:1038A0008C1F001050000010A026001000470010D0
:1038B0001C470010603D0010701F001018470010DA
:1038C0005E3D00108B4B1A888B4B1A838A4B01226A
:1038D0009A76894B0022DA76874B93F82F30012BAA
:1038E00032D1864BFF221A70844B03225A70834BCD
:1038F000FF229A70814BFF22DA70804BFF221A71EF
:103900007F4B9B68DAB27D4B5A717D4B9B681B0ADB
:10391000DAB27A4B9A717A4B9B681B0CDAB2774B0E
:10392000DA71774B1A7B764B597B08230193734BE3
:1039300000930B464FF46C410720FEF7EDFF034662
:10394000FB77002000F090FAFB68B3F56C4F40F075
:1039500007816C4B1B7B7A799A4240F00181BB68EE
:103960001B78102B40F0FC80BB6801331B789AB2A7
:10397000BB6802331B789BB21B029BB213443B8390
:103980005F4B1B78002B09D13B8B40F2F9629342CD
:1039900004D85B4B93F80C37012B35D1574BFF22E2
:1039A0001A70574BB3F80A3740F2F962934203D9C1
:1039B000524B02225A7002E0504B01225A704F4B78
:1039C000FF229A704D4BFF22DA704C4BFF221A7186
:1039D000BB685A79494B5A71BB689A79474B9A71BF
:1039E000BB68DA79454BDA7197F828107A790823A1
:1039F0000193424B00930B464FF46C410720FEF7B6
:103A00008BFF0346FB77ABE0BB6807331B781A04D8
:103A1000BB6806331B781B021344BA680532127860
:103A20001344374A9360364B9B6807F116021146E0
:103A30001846FFF767FA0346012B67D1304B012286
:103A40001A702F4B01225A702D4B01221A712C4AE9
:103A500097F8283013732A4A7B795373BB68DA7856
:103A6000274B9A73264B0022DA73BB6801331B780D
:103A70009AB2BB6802331B789BB21B029BB2134401
:103A80009AB21F4BA3F80A2700237B8309E07B8BA4
:103A9000BA681A447B8B1178184AD1547B8B013356
:103AA0007B837B8B072BF2D9144B11221A70134B9B
:103AB000DA78124B5A70114B01229A700F4BFF2289
:103AC000DA7097F828107A79082301930B4B00934A
:103AD0000B464FF46C410720FEF71EFF0346FB77B1
:103AE000094B1A88044B9A84034B012283F8262041
:103AF00036E000BF9E260010004700105000001066
:103B00008C1F00107C1F00106C1F0010734BFF22D5
:103B10001A70724B02225A70704BFF229A706F4BD0
:103B2000FF22DA706D4BFF221A71BB685A796B4B1A
:103B30005A71BB689A79694B9A71BB68DA79674B9D
:103B4000DA7197F828107A7908230193634B009370
:103B50000B464FF46C410720FEF7DEFE0346FB7771
:103B60005F4B1B78012B40F0B3805D4B5B78012BE2
:103B700040F0AE805B4B93F82730012B32D1002010
:103B800000F072F9554BFF221A70544B03225A7001
:103B9000524BFF229A70514BFF22DA704F4BFF229B
:103BA0001A714F4B9B68DAB24C4B5A714C4B9B6865
:103BB0001B0ADAB2494B9A71494B9B681B0CDAB26B
:103BC000464BDA71464B5A7B454B197B08230193D0
:103BD000424B00930B464FF46C410720FEF79CFECE
:103BE0000346FB77FB68B3F56B4F71D13C4B5B7BB6
:103BF0007A799A426CD13A4B1B7B97F828209A42EB
:103C000066D1394B1A88374B1A83BB681B78013B46
:103C10009BB21A46D200D31ABB8301237B830DE0EB
:103C20007B8BBA681A44BB8B591CB983194612782E
:103C30002B4B0B441A747B8B01337B837B8B072BC1
:103C4000EED9274BDB7B0133DAB2254BDA73244BF9
:103C5000DA7B234B9B7B9A423AD1204B13221A707A
:103C60001F4BB3F80A37DAB21C4B5A701B4B0022B9
:103C70009A701B4B9A7B194BDA70184BFF221A7102
:103C8000174B9B68DAB2154B5A71154B9B681B0A90
:103C9000DAB2124B9A71124B9B681B0CDAB20F4BC3
:103CA000DA710F4B5A7B0E4B197B082301930B4B98
:103CB00000930B464FF46C410720FEF72DFE0346A0
:103CC000FB77012000F0D0F8054B012283F80C2788
:103CD000FB7F18462037BD4680BD00BF5000001056
:103CE0008C1F001000470010603D001080B487B0AA
:103CF00000AF396011461A460346FB710B46BB7193
:103D000013467B710023FB757B79FF2B02D0354B6B
:103D1000FB6001E0344BFB60FB681B78002B04D197
:103D2000BB8C40F2F962934202D90123FB7552E049
:103D300000233B610CE03B693A6A13441978FA6846
:103D40003B69134410330A461A703B6901333B61E7
:103D5000BB8C3A699A42EEDBBB8C3B610CE03B6961
:103D6000B3F5DF6F0EDCFA683B6913441033FF22B2
:103D70001A703B6901333B61BB8C06333A699A4246
:103D8000EDDD00E000BFFB683A689A60FB68BA8C22
:103D9000A3F80A27FB68BA791A73FB687A795A7311
:103DA000BB8C3B61FB6800229A7308E03B69073BD0
:103DB0003B61FB689B7B0133DAB2FB689A733B691A
:103DC000002BF3DCFB680022DA73FB6802221A7016
:103DD000FB6801225A70FB7D18461C37BD4680BC2B
:103DE000704700BF8C1F00104836001080B582B0AD
:103DF00000AF0346FB71FB79002B1FD1164B00224D
:103E00001A70154B00225A70134B00229A70124BF5
:103E100000229A60104BFF221A730F4BFF225A7335
:103E20000D4B00229A730C4B0022DA730A4B0022CE
:103E3000A3F80A27084B002283F80C270748FEF74F
:103E4000B3FD0748FEF7B0FD064B01221A7000BF14
:103E50000837BD4680BD00BF48360010104700102F
:103E6000144700106600001080B582B000AF034612
:103E7000FB71FB79002B22D11F4B00221A701E4BC5
:103E800000225A701C4B0022DA701B4B00221A7160
:103E9000194B00229A60184BFF221A73164BFF220F
:103EA0005A73154B00229A73134B0022DA73124B8C
:103EB0000022A3F80A27104B002283F80C270F4892
:103EC000FEF772FD0E48FEF76FFD0E48FEF76CFD23
:103ED0000D48FEF769FD0D48FEF766FD0C48FEF73C
:103EE00063FD0C48FEF760FD0B4B01221A7000BF0A
:103EF0000837BD4680BD00BF8C1F0010184700105A
:103F00001C470010204700102447001028470010CD
:103F10002C470010304700106600001080B483B0BA
:103F200000AF064B1B79FB71044B00221A71FB7921
:103F300018460C37BD4680BC704700BF7C1F001080
:103F400080B483B000AF0346FB71FB7903F01F031D
:103F5000012202FA03F1054A97F907305B0942F89A
:103F6000231000BF0C37BD4680BC704700E100E065
:103F700080B487B000AF7860396000237B617B68D4
:103F8000012B01D1104B00E0104B3B610A23FB6079
:103F90000F4AFB68B2FBF3F23B68B2FBF3F3013B61
:103FA0007B617B69C3F309037B610A4AFB6852F8B2
:103FB00023307A6913437B613B697A695A6100BF98
:103FC0001C37BD4680BC7047004004400080044060
:103FD00040787D017083000080B584B000AF7860C8
:103FE00039607B68012B01D1264B00E0264BFB603A
:103FF0007B68012B17D1254BD3F8C430234A43F4F7
:104000000053C2F8C430224B1B68214A43F001031D
:1040100013601F4B1B681E4A43F0040313601920F2
:10402000FFF78EFF16E0194BD3F8C430174A43F45C
:104030008043C2F8C430164B1B68154A43F4007322
:104040001360134B1B68124A43F40063136019207A
:10405000FFF776FF0F4B02221A60FB6801221A60FD
:10406000FB6800221A61FB6800229A603968786850
:10407000FFF77EFFFB6803221A6100BF1037BD46C1
:1040800080BD00BF004004400080044000C00F40DD
:1040900000C0024000C0034080B485B000AF78602B
:1040A0007B68012B01D1064B00E0064BFB60FB68EF
:1040B00000221A6000BF1437BD4680BC704700BFA5
:1040C000004004400080044080B485B000AF7860B8
:1040D0007B68012B01D10A4B00E00A4BFB6000BF5B
:1040E000FB68DB6903F00403002BF9D07B68013B1C
:1040F000054A0121D15400BF1437BD4680BC70472A
:1041000000400440008004404004001080B487B0A8
:1041100000AFF860B9601346FB71FB68012B01D159
:10412000204B00E0204B7B61BB681B7B1B0403F42E
:104130007023BA68527B012A02D14FF0004200E09E
:1041400000221343BA68927B012A02D14FF08042C9
:1041500000E0002213433B617B69DB6903F0040349
:10416000002B1AD07B693A691A63BB681A687B69AD
:104170005A63BB6804331A687B699A63BB68083367
:104180001A687B69DA63FB79012B03D17B693122E1
:104190005A6002E07B6921225A6000BF1C37BD468D
:1041A00080BC7047004004400080044080B485B06B
:1041B00000AF786039607B68012B01D11B4B00E0B8
:1041C0001B4BFB60FB681B6ABB60BB68DB0FDBB291
:1041D0001A463B685A73BB6803F08043002B14BF38
:1041E00001230023DBB21A463B689A73BB681B0CA1
:1041F000DBB203F00F03DAB23B681A73FB685A6A4A
:104200003B681A603B689B7B002B09D13B680433F9
:10421000FA68926A1A603B680833FA68D26A1A60D0
:1042200000BF1437BD4680BC704700BF004004404B
:104230000080044080B582B000AF674B1B78012B33
:1042400040F09580654BDB687B607B6803F0010381
:10425000002B00F08480624B1B781A4613465B00EB
:104260001344DB005F4A134419460120FFF79EFF09
:1042700000BF5D4B1B78002BFBD0594B1B781946B8
:104280005A4B1878574A0B465B000B44DB0013442B
:104290000F3302461A70524B1B781946544B18784C
:1042A000504A0B465B000B44DB00134410330246BC
:1042B0001A704B4B1B7819464E4B1878494A0B46DF
:1042C0005B000B44DB001344113302461A70444B6D
:1042D0001B781946484B1878424A0B465B000B4442
:1042E000DB001344123302461A703D4B1B7819460B
:1042F000424B18783B4A0B465B000B44DB001344EF
:10430000133302461A70364B1B7819463C4B18780B
:10431000344A0B465B000B44DB0013441433024663
:104320001A702F4B1B781946364B18882D4A0B46AE
:104330005B000B44DB001344163302461A80284B03
:104340001B780133DAB2264B1A70254B1B78282BC9
:1043500002D1234B00221A70204B04225A607B6842
:1043600003F00203002B02D0274B01221A70274BC7
:104370001B78012B2CD1264BDB687B607B6803F01C
:104380000103002B1CD0234B1B781A4613465B00FD
:104390001344DB00204A134419460220FFF706FFAE
:1043A0001B4B04225A601B4B1B780133DAB2194BAA
:1043B0001A70184B1B78282B02D1164B00221A704A
:1043C0007B6803F00203002B02D00F4B01225A70CE
:1043D00000BF0837BD4680BD4204001000400440C5
:1043E00039040010643D0010450400106E000010F8
:1043F0006D0000106C0000104A0400104904001009
:10440000480400104604001040040010430400104B
:10441000008004403B0400102441001080B483B0AD
:1044200000AF78607B68012B09D10E4BDB6903F08C
:10443000C203002B01D100230FE001230DE07B68B4
:10444000022B09D1084BDB6903F0C203002B01D119
:10445000002302E0012300E0012318460C37BD468B
:1044600080BC7047004004400080044080B584B0A8
:1044700000AFF860B9601346FB71FB68012B03D0F5
:10448000FB68022B0AD013E0154B00221A70154B63
:1044900000221A70144B01221A700BE0134B0022F9
:1044A0001A70134B00221A70124B01221A7001E08D
:1044B000012311E0104AFB791370FB68BA681146BA
:1044C0001846FFF789FDFB681846FFF7E5FDFB6816
:1044D0001846FFF7F9FD002318461037BD4680BD8A
:1044E000390400103A040010420400103B0400108C
:1044F0003C04001043040010E444001090B486B063
:1045000000AFF860B9607A603B600123BB75FB685F
:10451000012B04D0FB68022B00F0AD80FEE0824B43
:104520001A78824B1B789A4200F0F5807E4B1B78FC
:1045300019467F4A0B465B000B44DB0013441B68A3
:104540001A46BB681A60784B1B781946784A0B46A6
:104550005B000B44DB0013440C331B781A463B68AA
:104560001A600023FB7513E06F4B1B781C46F97D26
:10457000FB7D7A681A446E4823465B002344DB00C7
:1045800003440B4404331B781370FB7D0133FB752C
:10459000FA7D3B681B689A42E6DB634B1B78194641
:1045A000634A0B465B000B44DB00134416331A8846
:1045B0003B6A1A805C4B1B7819465D4A0B465B00D0
:1045C0000B44DB00134414331A783B6A9A70564B41
:1045D0001B781946564A0B465B000B44DB0013441C
:1045E00013331A783B6ADA704F4B1B781946504ADE
:1045F0000B465B000B44DB00134412331A783B6A12
:104600001A71494B1B781946494A0B465B000B440B
:10461000DB00134411331A783B6A5A71424B1B7802
:104620001946434A0B465B000B44DB00134410332E
:104630001A783B6A9A713C4B1B7819463C4A0B46E8
:104640005B000B44DB0013440F331A783B6ADA71CA
:10465000354B1B780133DAB2334B1A70324B1B786F
:10466000282B02D1304B00221A70324B05221A60DF
:104670000023BB754FE0304B1A78304B1B789A42C1
:104680004BD02D4B1B7819462D4A0B465B000B4433
:10469000DB0013441B681A46BB681A60264B1B7864
:1046A0001946274A0B465B000B44DB0013440C33CE
:1046B0001B781A463B681A600023FB7513E01E4BFB
:1046C0001B781C46F97DFB7D7A681A441C482346FA
:1046D0005B002344DB0003440B4404331B7813705A
:1046E000FB7D0133FB75FA7D3B681B689A42E6DB74
:1046F000114B1B780133DAB20F4B1A700E4B1B783B
:10470000282B02D10C4B00221A700A4B05221A608A
:104710000023BB7501E000BF00E000BFBB7D184671
:104720001837BD4690BC70473A0400103904001099
:10473000643D0010E64400103C0400103B040010EF
:104740002441001080B586B000AFF860B960134610
:10475000FB710123FB75FB68013B194AD35C002BFD
:104760001CD0FB68013B164A0021D154FB68FA7942
:10477000B9681846FFF7CAFC0023FB7508E0F86823
:10478000FFF74CFE0346012B02D10123FB7505E028
:10479000FB68013B0A4AD35C002BF0D0FB7D002B69
:1047A00009D1FB68012B03D1064B05221A6002E0F8
:1047B000044B05221A60FB7D18461837BD4680BDA4
:1047C00040040010E644001080B58CB000AFF860E3
:1047D000B9607A603B60FB68012B04D0FB68022B58
:1047E00001D001232EE0BB687B61002387F82F30C6
:1047F00010E097F82F307A681A4497F82F30127823
:1048000007F130010B4403F8182C97F82F300133CF
:1048100087F82F3097F82F30072BEAD93B68DBB2A7
:1048200087F82030094B1B7887F82130002387F860
:10483000223097F8382007F114031946F868FFF77B
:1048400081FF034618463037BD4680BDE444001062
:1048500080B483B000AF78607B68002B03D1074B36
:10486000074A1A6005E07B68012B02D1034B054A19
:104870001A6000BF0C37BD4680BC7047680000104E
:1048800090D0030020A1070080B485B000AF03469C
:10489000FB710023FB60FB79042B1CD801A252F8AA
:1048A00023F000BFB9480000BF480000C548000021
:1048B000CB480000D14800000A4BFB600CE00A4BDB
:1048C000FB6009E0094BFB6006E0094BFB6003E07D
:1048D000084BFB6000E000BFFB6818461437BD467C
:1048E00080BC704700C0092020C0092040C00920BA
:1048F00060C0092080C0092080B584B000AF0346A5
:104900003960FB711346BB71FB791846FFF7BCFF9A
:10491000F860FB68002B10D0BB79002B06D0FB6839
:104920001A683B681A43FB681A6006E0FB681A685D
:104930003B68DB431A40FB681A6000BF1037BD4676
:1049400080BD80B584B000AF03463960FB71FB7950
:104950001846FFF799FFF860FB68002B02D0FB6850
:104960003A689A6100BF1037BD4680BD80B584B0FB
:1049700000AF03463960FB71FB791846FFF784FFEF
:10498000F860FB68002B02D0FB683A68DA6100BF70
:104990001037BD4680BD80B584B000AF0346FB71C3
:1049A000FB791846FFF770FFF860FB68002B02D018
:1049B000FB685B6900E0002318461037BD4680BDE8
:1049C00080B487B000AF0346FB710B46BB71134642
:1049D0007B71BB797B61FB795B003B61174BFB60B3
:1049E0007B690F2B05D97B69103B7B613B690133E8
:1049F0003B613B699B00FA68134419687B695B0063
:104A0000032202FA03F3DA433B699B00F86803448C
:104A10000A401A603B699B00FA68134419687A7966
:104A20007B695B009A403B699B00F86803440A433A
:104A30001A6000BF1C37BD4680BC704700C00240F2
:104A400080B487B000AF0346FB710B46BB711346C1
:104A50007B71BB797B61FB795B003B61174BFB6032
:104A60007B690F2B05D97B69103B7B613B69013367
:104A70003B613B699B00FA68134419687B695B00E2
:104A8000032202FA03F3DA433B699B00F86803440C
:104A90000A401A603B699B00FA68134419687A79E6
:104AA0007B695B009A403B699B00F86803440A43BA
:104AB0001A6000BF1C37BD4680BC704740C0024032
:104AC00080B485B000AF0346FB710B46BB71134643
:104AD0007B71144BFB607B79012B0ED1FB799B0022
:104AE000FA6813441968BB7901229A40FB799B004C
:104AF000F86803440A431A600FE0FB799B00FA68E8
:104B000013441968BB79012202FA03F3DA43FB79F3
:104B10009B00F86803440A401A6000BF1437BD4682
:104B200080BC704768C0024080B582B000AF78603A
:104B30007B6818787B6859787B689B781A46FFF702
:104B40003FFF7B6818787B6859787B68DB781A466A
:104B5000FFF776FF7B6818787B6859787B681B794C
:104B60001A46FFF7ADFF00BF0837BD4680BDFFFF07
:104B700080B500AF00F088F800F0AAFB4FF000709D
:104B800000F0EBF80346012B04D14FF4E12000F0D4
:104B90003FFD03E04FF4E13000F03AFD00F05CF936
:104BA000324B00221A70324B00221A7000F050FF74
:104BB000304B00221A70304B01221A702F4B4FF4E9
:104BC0007A721A80FBF79CFB03212D4800F02CFF22
:104BD000FBF7E2FB2B4B00221A704FF0807000F0C5
:104BE000BCF80346012B03D1264B01221A7002E0C8
:104BF000244B00221A701F4B1B78012B03D100F0AD
:104C000099F800F0E7FF1E4BDB78012BE0D1032180
:104C10001B4800F009FF154B1B78002B0BD0134BE2
:104C20001B78013BDAB2114B1A704FF4800101205E
:104C3000FFF79CFE04E04FF480010120FFF781FEA6
:104C40000B4B1B78002B0BD0094B1B78013BDAB2C6
:104C5000074B1A704FF400010120FFF787FEB7E7FA
:104C60004FF400010120FFF76CFEB1E7E5440010AE
:104C7000E6440010350600103D0D0010681F0010BE
:104C8000004700104404001080B582B000AF00233C
:104C9000BB7000233B710023FB7001233B70122388
:104CA0007B703B461846FFF73FFF16237B703B4661
:104CB0001846FFF739FF17237B703B461846FFF76E
:104CC00033FF01233B7018237B703B461846FFF7E8
:104CD0002BFF19237B703B461846FFF725FF1A234D
:104CE0007B703B461846FFF71FFF01224FF444013B
:104CF0000120FFF701FE00224FF0E0610120FFF7E5
:104D0000FBFD00F004F800BF0837BD4680BD80B54C
:104D100000AF4FF400010120FFF713FE4FF48001B4
:104D20000120FFF70EFE4FF480210120FFF709FE5E
:104D300000BF80BD80B500AF4FF400010120FFF738
:104D400015FE4FF480010120FFF710FE4FF4802183
:104D50000120FFF70BFE00BF80BD80B584B000AF1F
:104D600078600120FFF717FEF860FA687B6813404F
:104D7000BB60BB68002B01D1012300E00023184673
:104D80001037BD4680BDFFFF80B483B000AF03463F
:104D9000FB71FB7903F01F03012202FA03F1054ABC
:104DA00097F907305B0942F8231000BF0C37BD4666
:104DB00080BC704700E100E080B400AF1D4B0022D2
:104DC0001A701D4B1B78DBB21B4A43F00103DBB2A8
:104DD00013701A4B00221A80174B93F82030DAB266
:104DE000174B1A70144B93F82430DAB2154B1A7023
:104DF000114B93F82830DAB2134B1A700E4B93F81C
:104E00002C30DAB2114B1A700B4B93F83830DAB2FF
:104E10000F4B1A70084B9B8F9BB2DBB23033DAB268
:104E20000C4B1A70034B01221A7000BFBD4680BCA8
:104E3000704700BF450400100040024046040010C7
:104E400048040010490400104A0400106C000010CF
:104E50006D0000106E00001080B500AF0F4BD3F84E
:104E6000C4300E4A43F40073C2F8C4300C4B122213
:104E70001A720B4B00221A64094B00221A74084B59
:104E800001221A73064B01221A72054B01221A7075
:104E90001120FFF779FF00BF80BD00BF00C00F40A9
:104EA0000040024080B483B000AF7860134A7B6852
:104EB0001B7882F82030114A7B685B7882F82430B6
:104EC0000E4A7B689B7882F828300C4A7B68DB7836
:104ED00082F83030094A7B681B7982F82C30074A07
:104EE0007B685B7982F83830044A7B68DB8893877B
:104EF00000BF0C37BD4680BC704700BF0040024079
:104F000080B483B000AF7860164B93F82030DAB2EB
:104F10007B681A70134B93F82430DAB27B685A70AE
:104F2000104B93F82830DAB27B689A700D4B93F8E7
:104F30003030DAB27B68DA700A4B93F82C30DAB290
:104F40007B681A71074B93F83830DAB27B685A7174
:104F5000044B9B8F9AB27B68DA8000BF0C37BD464A
:104F600080BC70470040024080B483B000AF03466D
:104F7000FB71FB7903F01F03012202FA03F1054ADA
:104F800097F907305B0942F8231000BF0C37BD4684
:104F900080BC704700E100E080B483B000AF2E4BCE
:104FA0009B68BB71BB7903F00403002B24D02A4B10
:104FB0001B7DFB711BE0284B1B787B71FB7903F099
:104FC0008E03002B05D0FB7903F08E03234A136078
:104FD0000AE0234BD3F800315A1C2149C1F80021C3
:104FE000DBB21F497A79CA541B4B1B7DFB71FB79DD
:104FF00003F00103002BDED1BB7903F00203002B89
:105000001CD0184BD3F80021164BD3F80431D31A17
:10501000DBB2002B0FD0134BD3F804315A1C1149CB
:10502000C1F80421DBB20C4A0E49CB5C13700E4B65
:1050300000221A7002E00C4B01221A70064B1B7DF5
:10504000DBB29BB203F01E039AB2084B1A8000BF7A
:105050000C37BD4680BC704700C00040E8440010DB
:10506000EC440010F8450010F4450010F64500101F
:1050700080B586B000AFF860B9601346FB710123BC
:10508000FB750521234800F0CFFC03E0224B1B7881
:10509000012B05D0214B93F83730002BF6D000E0E0
:1050A00000BF1E4B93F83730002B2ED100233B61FD
:1050B00010E0FB685A1CFA60194AD2F80021511C12
:1050C0001748C0F80011D2B21978154B99543B69B2
:1050D00001333B613B69BA689A42EAD80E4B002221
:1050E0001A700F4BD3F804315A1C0D49C1F8042132
:1050F000DBB20C4A0A49CB5C1370FB79012B02D15D
:10510000094B05221A700023FB75FB7D18461837E2
:10511000BD4680BD34470010F44500100047001024
:10512000F845001000C00040E544001080B586B08E
:1051300000AFF860B9601346FB71304B1B78002B51
:1051400027D10A212E4800F06FFC00F005FF03462E
:10515000B3F1FF3F16D004E02A4B93F83730012B10
:1051600006D000F0F9FE034613F1020FF4D000E080
:1051700000BF244B93F83730002B03D1B968F8688F
:1051800000F0BEFEFB79012B34D11F4B05221A70B3
:1051900030E0BB68B3F5807F06D8FB791A46B96862
:1051A000F868FFF765FF25E0BB687B6100233B6182
:1051B000FA683B691344FA794FF480711846FFF797
:1051C00057FF0346012B14D07B69A3F580737B61E5
:1051D0003B6903F580733B617B69B3F5807FE7D85A
:1051E000FA683B691344FA7979691846FFF740FF7A
:1051F00000E000BF00BF1837BD4680BD440400106A
:105200003447001000470010E544001080B588B016
:1052100000AFF860B9601346FB710023FB61294BB6
:105220001B78002B06D1BB681946F86800F03AFEDF
:10523000F86138E0244BD3F80021234BD3F8043134
:10524000D31ADBB2002B2ED01F4BD3F800211E4BFC
:10525000D3F80431D31ADBB27B617B69002B22DDEA
:105260000023BB6119E0184BD3F804315A1C1649CE
:10527000C1F80421DAB2F968FB690B4412498A5C6F
:105280001A70BB68013B1A46FB6993420AD0FB695E
:105290000133FB61BB690133BB617B69BA699A4227
:1052A000E1D300E000BFFB69002B05D0FB79012BA7
:1052B00002D1064B05221A70FB6918462037BD46FD
:1052C00080BD00BF44040010EC440010E544001011
:1052D00080B500AF00F0DAFC00BF80BD90B585B0AE
:1052E00000AFC7E90001D7E9000102F08DFE0346D7
:1052F000FB60F86802F0CBFE03460C461A462346D4
:10530000D7E9000102F0CCFE0346002B01D00123B7
:1053100000E0002318461437BD4690BD90B589B013
:1053200000AFC7E902017A603B60374BFB610023A5
:105330007B615FE0354A7B6952F82330184602F002
:1053400087FF03460C461A462346D7E9020102F0BE
:10535000E5FE0346002B17D02C4A7B6952F8233018
:10536000184602F075FF03460C461A462346D7E955
:10537000020102F0C9FC03460C461846214602F021
:105380001BFE0346BB6112E0204A7B6952F82330C2
:10539000184602F05DFFD7E9022302F0B5FC034690
:1053A0000C461846214602F007FE0346BB6116492B
:1053B000F86902F069FF0346002B16D1F969B86954
:1053C00002F071FF0346002B0FD07B69013B104AAE
:1053D00052F823207B681A607B69013B0D4A52F822
:1053E00023203B681A60002309E0BB69FB617B69ED
:1053F00001337B617B69472B9CDD4FF0FF331846FF
:105400002437BD4690BD00BF000080BF7000001073
:1054100090010010B00200102DE9B0438CB000AF35
:10542000F860B9607A603B60F86802F030FE0446CC
:105430000D46B86802F02BFE4FF00002724B02F0EE
:105440003DFB02460B462046294602F0BDFB0346C3
:105450000C46C7E908344FF000036C4CC7E90A3426
:10546000D7E90801FFF73AFF0346002B10D0D7E930
:10547000080102F0C9FD02467B681A603B684FF0E4
:1054800000021A60BB6C4FF07E521A600023A3E04A
:10549000F86802F0FCFD04460D46B86802F0F7FD1E
:1054A0004FF00002584B02F009FB02460B46104633
:1054B0001946D7E90A2302F001FB02460B462046B3
:1054C000294602F081FB03460C461846214602F0AD
:1054D0009BFD0346FB61F86802F0D9FD04460D46CA
:1054E000B86802F0D4FD4FF00002474B02F0E6FA34
:1054F00002460B4690469946F86902F0C8FD0246FE
:105500000B464046494602F0D9FA02460B46204671
:10551000294602F059FB03460C46C7E9043432A37E
:10552000D3E90023D7E9040102F04AFE0346002B29
:1055300009D02FA3D3E90023D7E9040102F0C5FD68
:105540000346002B3DD14FF00002304BD7E90A0152
:1055500002F00DFE0346002B1AD027A3D3E9002347
:10556000D7E90A0102F0D0FB03460C46C7E90A342A
:105570001DA3D3E90023D7E90A0102F0A6FD0346E3
:10558000002B1DD01EA4D4E90034C7E90A347FE7FC
:1055900019A3D3E90023D7E90A0102F089FC0346E5
:1055A0000C46C7E90A3412A3D3E90023D7E90A015C
:1055B00002F006FE0346002B02D04FF0FF330BE053
:1055C00066E700BF7B68FA691A60BB6C3A68D7E986
:1055D0000401FFF7A3FE034618463037BD46BDE879
:1055E000B08300BFAFF300809A9999999999F13FE0
:1055F000666666666666FE3FFCA9F1D24D62503F64
:1056000071AC8BDB6800F83F000030400000F83FD1
:1056100090B589B002AF7860444B0022C3F80021F6
:10562000424BD3F80031414AC2F80431404B0022CA
:10563000C3F800213E4BD3F800313D4AC2F8043193
:105640003C4B7B6107F10C0107F1100207F10803E5
:1056500000930B4679687869FFF7DEFE0346B3F1E5
:10566000FF3F02D14FF0FF335BE0334BD3F8C43040
:10567000314A43F00803C2F8C4302F4BD3F8A831A5
:105680002D4A23F0C003C2F8A8312B4BD3F8A83120
:10569000294A43F04003C2F8A831284B1B68274A27
:1056A00023F0F0031360254B1B68244A43F050039A
:1056B0001360234B83221A733B69002B00DAFF33FC
:1056C0001B121A461E4BD2B21A713B695A42DBB208
:1056D000D2B258BF53421A4ADBB21370BB681846A5
:1056E00002F09AFD03461B015CB2FB68184602F00B
:1056F00093FD03465BB223435AB2114BD2B283F8F7
:1057000028200F4B03221A730D4B03225A600C4BB7
:1057100007221A720B4B01221A700520FFF724FC96
:10572000002318461C37BD4690BD00BFF845001049
:10573000EC44001000D8B80500C00F4000C0024083
:1057400000C00040F445001080B400AF4B4B202255
:10575000C3F8A02100BF494BD3F8A03103F04003A8
:10576000002BF8D0454B0322C3F80421434B002201
:10577000C3F8A821414B0022C3F8AC213F4B0122C2
:10578000C3F80C213D4B3E4AC3F884203B4BAA2270
:10579000C3F88C20394B5522C3F88C20374B01229B
:1057A000C3F88020354BAA22C3F88C20334B5522F6
:1057B000C3F88C2000BF314BD3F8883003F08063EE
:1057C000002BF8D02D4B0322C3F880202B4BAA22AC
:1057D000C3F88C20294B5522C3F88C2000BF274BDF
:1057E000D3F8883003F04073002BF8D0234B2322EA
:1057F000C3F8A420214BAA22C3F8AC201F4B55228A
:10580000C3F8AC201D4B0122C3F8A0201B4BAA22D9
:10581000C3F8AC20194B5522C3F8AC2000BF174B7E
:10582000D3F8A83003F48063002BF8D0134B032285
:10583000C3F8A020114BAA22C3F8AC200F4B55226D
:10584000C3F8AC2000BF0D4BD3F8A83003F440736D
:10585000002BF8D0094B0B4AC3F8C420074B002299
:10586000C3F8C821054B1B6823F47043034A43F473
:105870008043136000BFBD4680BC704700C00F402E
:1058800063000500DE87280480B483B000AF0346C0
:10589000FB71FB7903F01F03012202FA03F1054AB1
:1058A00097F907305B0942F8231000BF0C37BD465B
:1058B00080BC704700E100E080B483B000AF0023FB
:1058C0007B6026E0554A7B689B0013449B78012B44
:1058D0001CD1524A7B689B001344DB78002B15D106
:1058E0004E4A7B6832F82330013B99B24B4A7B68C1
:1058F00022F82310494A7B6832F82330002B05D167
:10590000464A7B689B0013440122DA707B680133AE
:105910007B607B680D2BD5DD00237B6042E0404936
:105920007A6813465B001344DB000B4416331B7884
:10593000012B34D13A497A6813465B001344DB00EB
:105940000B4414331B78002B29D135497A68134650
:105950005B001344DB000B4412331B88013B98B2FD
:105960002F497A6813465B001344DB000B44123363
:1059700002461A802A497A6813465B001344DB000A
:105980000B4412331B88002B09D125497A68134632
:105990005B001344DB000B44143301221A707B6854
:1059A00001337B607B68632BB9DD00237B602CE0D7
:1059B0001C497A6813469B001344DB000B441B7898
:1059C000012B1FD117497A6813469B001344DB0053
:1059D0000B440A331B88002B14D012497A681346F3
:1059E0009B001344DB000B440A331B88013B98B235
:1059F0000C497A6813469B001344DB000B440A33BE
:105A000002461A807B6801337B607B68632BCFDDA5
:105A100000BF0C37BD4680BC704700BF0047001078
:105A200040150010A426001080B483B000AF786049
:105A30000B467B807B687A881A807B6801229A708B
:105A40007B680022DA7000BF0C37BD4680BC70470F
:105A500080B582B000AF1D4B00221A8000237B600E
:105A600013E01B4A7B68002122F82310184A7B6848
:105A70009B00134400229A70154A7B689B001344D4
:105A80000022DA707B6801337B607B680D2BE8DDD8
:105A9000104BD3F8C4300F4A43F48033C2F8C430FB
:105AA0000C4BD3F8AC310B4A43F04063C2F8AC3135
:105AB000094B43F2D4021A60074B0A221A721D20C6
:105AC000FFF7E2FE00BF0837BD4680BD3847001033
:105AD0000047001000C00F4000000B4080B500AF31
:105AE000134B1B7ADBB2124A43F00103DBB2137291
:105AF000FFF7E2FE0F4B1B889BB2002B06D00D4B2D
:105B00001B889BB2013B9AB20A4B1A800A4B1B7846
:105B1000012B0BD1094B1B8840F2E632934205D88A
:105B2000064B1B8801339AB2044B1A8000BF80BD1C
:105B300000000B40384700104504001046040010D8
:105B400080B400AF72B6224B0122C3F88020204BF4
:105B5000AA22C3F88C201E4B5522C3F88C2000BF0C
:105B60001B4BD3F8883003F00073002BF8D1184B8F
:105B70000022C3F88020164BAA22C3F88C20144BB5
:105B80005522C3F88C2000BF114BD3F8883003F0A6
:105B90008073002BF8D10E4B1B680D4AC3F30B0327
:105BA00013600B4B1B680A4A43F4A0431360084B75
:105BB0000022C3F80421064B0022C3F80C21044B39
:105BC0000022C3F8A02100BFBD4680BC704700BFC3
:105BD00000C00F4080B500AFFFF7B2FF72B6064BB2
:105BE000064A1A60064B39221A60034B1B680549A6
:105BF0000348984700BF80BDD4030010F11FFF1F6A
:105C00003C4700105047001030B583B000F0ECF96D
:105C10000E4C01250095204600211D22082300F08E
:105C200067FB0095204600211E22082300F060FB40
:105C30001222074BC3F8F42F054BD3F8F83F03F0BB
:105C40001203122BF8D103B030BD00BF00C00240D8
:105C500000C0005008B5044B1B681B68DB68034A92
:105C60001068984708BD00BFD80300104C0400100E
:105C700006E04278042A02D142798A4204D01844CC
:105C80000378002BF5D10020704700BF10B598B005
:105C900000F0A0F9FFF7B8FF07A80021442201F0A7
:105CA000A0FC1E4B079303238DF828301C4B089350
:105CB0004FF4006309931B4B02931B4B03931B4B45
:105CC00005930493002306930123009318480221AF
:105CD0000922082300F00CFB164B1B681B685B684D
:105CE000154802A907AA9847044698B9124B1868A4
:105CF00002A907AA00F080F8044658B94FF0807254
:105D00000E4B1A600B4B1B681B689B680A4A106895
:105D100001219847204618B010BD00BF00C20050B6
:105D200000C00720948400005C840000DC030010A5
:105D300000C00240D80300104C04001000E100E055
:105D4000032A05D10B8A23F001031B041B0C0B82D1
:105D50000020704738B50C46022A02D0042A2CD005
:105D60003DE0204B1B681B685B6C0121A2689847D3
:105D700080B2E081638A03F004039BB263B1638A5B
:105D800023F004031B041B0C638240B3638A9BB2A1
:105D900043F00203638222E0638A03F008039BB2AC
:105DA000EBB1638A23F008031B041B0C6382638A34
:105DB0009BB243F00103638211E04B8A03F00603B8
:105DC0006BB9084B1B681B689D6C0121A2684FF4DE
:105DD0000073A847638A9BB243F0040363820020E8
:105DE00038BD00BFD80300104FF48072014B1A82F7
:105DF0000020704764470010F0B593B006460F4688
:105E00001546234C44F8040B68460021482201F053
:105E1000E8FB6B680093AB680193F8680221FFF719
:105E200027FF0290F8680A21FFF722FF0390194B21
:105E30000F93194B1B685B695B68304669462246C5
:105E40009847034608BB009A114B9A6002F500720E
:105E50000092019AA2F5007201920F4A12685268EC
:105E60005468304603210D4AA047034648B90A4BFF
:105E70001B685B685C6830460221094A044BA047F6
:105E80000346009A6A60019AAA60184613B0F0BDF2
:105E900064470010E95D0000D8030010415D000078
:105EA000555D000038B5144BDC8914B3A14228BFFE
:105EB00021468CB21D469968224601F090FBAB89C1
:105EC00023449BB2AB814FF080710C4AC2F8801022
:105ED000EA89934208D36B8A23F002031B041B0C4C
:105EE0006B820023EB81AB814FF08072034B1A6011
:105EF00000E00024204638BD6447001000E100E0C7
:105F000070B5124C248A04F48074A4B2D4B10F4B3F
:105F10001B8A13F0010F17D10B4602460B49088A62
:105F200080B240F001000882094C4FF08075C4F83F
:105F30008050084800680068066D08688121B047F5
:105F4000256070BD002070BD002070BD644700104A
:105F500000E100E0D8030010094B1B8A03F48073B2
:105F60009BB233B1064B1B8A13F0010F04D1002002
:105F700070474FF0FF3070476FF00100704700BF6F
:105F80006447001080B400AF074BD3F8A83003F487
:105F90008063002B14BF01230023DBB21846BD46EB
:105FA0005DF8047B704700BF00C00F4080B400AFB5
:105FB000074BD3F8A83003F40073002B14BF012360
:105FC0000023DBB21846BD465DF8047B704700BF76
:105FD00000C00F4080B500AF00F07EF90246014BD3
:105FE0001A6080BDD003001080B500AF01200321EE
:105FF000012200F0B3F80120012100F08DF800BF6C
:10600000FFF7C0FF034683F00103DBB2002BF7D19B
:106010000120032100F080F800BFFFF7C7FF03460F
:1060200083F00103DBB2002BF7D11F2000F0C2F890
:1060300080BD00BF80B400AF074BD3F8883003F0B9
:106040008073002B14BF01230023DBB21846BD462A
:106050005DF8047B704700BF00C00F4080B400AF04
:10606000074BD3F8883003F00073002B14BF0123D3
:106070000023DBB21846BD465DF8047B704700BFC5
:1060800000C00F4080B483B000AF0346FB71094AE3
:10609000FB795B0113448833AA225A60054AFB79D5
:1060A0005B011344883355225A600C37BD465DF8B6
:1060B000047B704700C00F4080B400AF054BD3F89D
:1060C0000C31DBB203F00303DBB21846BD465DF8CA
:1060D000047B704700C00F4080B400AF1846BD4637
:1060E0005DF8047B704700BF80B400AF1846BD4622
:1060F0005DF8047B704700BF80B400AF00231846F2
:10610000BD465DF8047B704780B500AF00F08CF8A9
:106110000346184680BD00BF80B584B000AF03467B
:106120003960FB710C4AFB7904335B0113441B6833
:10613000FB60FA683B681343FB60074AFB79043352
:106140005B011344FA681A60FB791846FFF79AFF5F
:106150001037BD4680BD00BF00C00F4080B586B07F
:1061600000AF0346B9607A60FB73FB7B002B05D15F
:106170007B681A04BB6813437B6104E07B685A01A7
:10618000BB6813437B610A4AFB7B04335B01134406
:106190007A695A60064AFB7B04335B01134401228F
:1061A0001A60FB7B1846FFF76DFF1837BD4680BDB0
:1061B00000C00F4080B485B000AF0346FB71FB798F
:1061C000FB600849074BD3F8C430FA68012000FA95
:1061D00002F21343C1F8C4301437BD465DF8047BA6
:1061E000704700BF00C00F4080B582B000AFFFF71E
:1061F00035FF0346002B02D00123FB7101E0002391
:10620000FB71FB7918460837BD4680BD80B400AFEE
:10621000044BD3F80431DBB201331846BD465DF8B8
:10622000047B704700C00F4080B500AFFFF744FF0C
:106230000346012B07D0022B09D0002B0BD1FFF70F
:1062400053FF034608E0FFF747FF034604E0FFF76C
:1062500053FF034600E00023184680BD80B584B09C
:1062600000AF0023FB60FFF7E5FE0346002B18D0CC
:106270000E4BD3F88430C3F30E030133BB600B4BDA
:10628000D3F884301B0CDBB201337B60FFF73CFF9B
:106290000246BB6803FB02F35A007B68B2FBF3F3D0
:1062A000FB60FB6818461037BD4680BD00C00F403C
:1062B00080B500AFFFF798FF0346002B05D0012BF8
:1062C00007D1FFF7CBFF034604E0FFF7ADFF03461E
:1062D00000E00023184680BD98B500AFFFF7E8FF47
:1062E0000446FFF793FF0346B4FBF3F3184698BD4B
:1062F00080B487B000AFF8607B600B46FB7213463A
:10630000BB72BB7A03F00F03DBB25B00FB75FB7A59
:106310005B00DAB2BB7A1B09DBB21344BB75BA7DF2
:10632000FB6853F82220FB7D032101FA03F3DB43D2
:1063300013403B61BA7D97F82010FB7D01FA03F30F
:1063400019463B691943FB6843F82210BA7DFB6884
:10635000103253F82220FB7D032101FA03F3DB43C3
:1063600013403B61BA7DFB7D796899403B691943D5
:10637000FB68103243F822101C37BD465DF8047BE1
:10638000704700BF034600F00F0040001B0648BFE7
:1063900001307047436810229A6019611A68D2066A
:1063A000FCD5704738B504461546FFF7F3FF204685
:1063B0002946BDE83840FFF7EDBF38B5044608462A
:1063C0001546FFF7DFFF010441F4A0612046FFF707
:1063D000E1FF20462946BDE83840FFF7DBBF4368B0
:1063E00030229A6019611A689206FCD55869704784
:1063F0004FF40C707047FFFF044A0029D0F8C80121
:10640000034908BF4FF48072FFF7CCBF00010100C1
:106410000005FE00D0F8C83100225B689A64D0F80D
:10642000A021D179D96401219964D279DA641A68FA
:10643000D205FCD54FF0FF329A635A639A600C2262
:106440005A6070470346B3F89E31D0F8C8019B07E5
:1064500003D50249024AFFF7A5BF70470005FE00B9
:10646000000101007047FFFF70B50904D0F8C86152
:10647000084D41F4000444F4807430462946224615
:10648000FFF790FF304629462246BDE87040FFF7EF
:1064900089BF00BF0005D00093682DE9F041B3F536
:1064A0000C7F8046144633D3566806F110026260B2
:1064B000A3F11002A2606568AA0702D001356560E9
:1064C000F9E705F50772A3F50B736260A3606368D3
:1064D00013F0030702D001336360F8E72846224631
:1064E00000F0E2FF39461022304601F07AF82368C6
:1064F000B5602846C5F8C8617360FFF78BFF284672
:106500003946FFF7B1FFC8F800503846BDE8F081C2
:106510000148BDE8F08100BF0A00040010B50A4A36
:10652000D0F8C841002908BF4FF4807220460749BF
:10653000FFF738FF636803225A641A68D205FCD556
:106540004FF480729A6010BD000101000005D80070
:1065500038B5054688780C46FFF714FF012102463E
:106560009140D5F8C8315B68586C014359649A640E
:10657000A288DA641A68D205FCD54FF480729A605A
:1065800038BD704710B504460846FFF7FBFE01040E
:1065900041F48001D4F8C80141F4A0614FF4807245
:1065A000BDE81040FFF7FEBE10B504460846FFF7F1
:1065B000E9FE010441F48001D4F8C80141F4A0616E
:1065C000024ABDE81040FFF7EDBE00BF0001200009
:1065D00010B504460846FFF7D5FE010441F48001DA
:1065E000D4F8C80141F4A0614FF48072BDE81040B6
:1065F000FFF7D8BE10B504460846FFF7C3FE0104F6
:1066000041F48001D4F8C80141F4A061024ABDE818
:106610001040FFF7C7BE00BF0001010010B50446DF
:106620000846FFF7AFFE010441F48001D4F8C80129
:1066300041F4A0614FF48072BDE81040FFF7B2BE94
:10664000043A38B51D46D0F8C8410D2A48D8DFE8CD
:1066500002F00E0E474747474747474744074A0A55
:106660000122002041E04FF4007200203DE0084686
:10667000FFF788FE012303FA00F0236815B11843E1
:10668000206002E023EA000020602268236821687D
:10669000DB071B4B02F0020201EA030348BF42F092
:1066A00004020BB142F020022168164B0B400BB1E3
:1066B00042F0400223681449194009B142F008022F
:1066C00023681249194009B142F010021204204611
:1066D0000F4942F48072FFF765FE0022104604E085
:1066E00000220C4801E00822002061684B6815B1C7
:1066F0001A434A6038BD23EA02024A6038BD00BF2F
:10670000200882A01004415008822008044110048F
:106710000005F30001000400D0F8C80101F00F03E8
:106720002DE9F0419B00456843F00103AB622C6A00
:106730002605FCD514F480681DD0C4F309085FEA6F
:10674000980C25D016460023AF690133634546F8FF
:10675000047BF9D102EB830204F003045CB1AE695F
:106760001444002326FA03F502F8015BA24203F168
:106770000803F7D1456841F248230B410022DB07AB
:10678000AA6202D4034AFFF718FE4046BDE8F08132
:106790004446E3E70005F200704700207047002000
:1067A0007047FFF7B9BFFFFFD0F8C8012DE9F041EE
:1067B00001F00F044668A400DF1C44F00204BF0887
:1067C000B4629846736206D0002452F8045B013428
:1067D000BC42F561F9D10023B362034AFFF7EDFD36
:1067E0004046BDE8F08100BF0005FA002DE9F04702
:1067F000D0F8C8918246D9F80420136823F0040128
:106800009160516801EA030818F0080461D118F09A
:10681000040F2BD0166B3EB3274605460121A1403D
:10682000314219D00F43916313689806FCD5E307F2
:1068300050693DD4002C00F09080AB6D63B1D9F865
:106840000020114201D0C1066DD402225046D5F875
:10685000D8109847D9F804201F2C05D0B74204F16E
:10686000010405F10405D9D10423936018F4007FD5
:106870000FD0DAF83C3063B148464049FFF78AFD53
:106880003F494846FFF7ABFDDAF83C300146504639
:10689000984718F0010F09D0DAF834300BB15046A0
:1068A0009847D9F80C300133C9F80C30BDE8F087AF
:1068B000AB6D002BD0D0D9F80020114201D0C20618
:1068C00029D403225046D5F8D8109847D9F8042087
:1068D000C2E748462B49FFF75DFD48462A49FFF7C6
:1068E0007EFDC606044626D4A50706D5DAF838305C
:1068F0001BB1504604F00101984704F00903092B2D
:10690000D4D1640724D5DAF82C30002BCED05046F1
:106910009847BDE8F08705225046D5F8D81098472B
:10692000D9F8042098E704225046D5F8D8109847A3
:10693000D9F8042090E75046FFF76CFD504600F070
:106940009DFCDAF82830002BCED050469847CBE794
:10695000DAF83030002BDAD1A8E743077FF56DAFC6
:10696000DAF85830002B3FF479AF01225046DAF8BC
:10697000D8109847D9F8042070E700BF0005FB0045
:106980000002FB000005FE000002FE0070B54D781D
:106990001646042D1A4618D003D84DB1022D0DD03D
:1069A00027E0222D13D0232D13D0202D21D115E047
:1069B0000BB3036A1BB33168984770BDDBB1846ABF
:1069C000DCB149883268A04770BD036B02E0436BBD
:1069D00000E0836B9BB14988984770BD2BB1C36BB6
:1069E0006BB100F11001984770BD00F110043460E4
:1069F00001E0044870BD104670BD204670BD1846C9
:106A000070BD00BF02000400012A38B504460846E4
:106A100002D0022A2AD04AE094F8143203F07F020E
:106A2000212A44D194F81822097E914202D0417E55
:106A300091423CD104F5EA72DB09C4F8CC2104F59B
:106A4000057104F5E67207D1456CA847054678BB89
:106A5000B4F81A3263BB26E0056C04F5E873A84766
:106A6000054628BB204600F098FB21E094F814323C
:106A700003F07F03212B1AD194F818320A7E9A4230
:106A800002D04A7E9A4212D1D4F8CC21B4F81A32FC
:106A9000456CD21AC4F8CC2104F5057104F5E672F0
:106AA000A847054620B9204600F0A0FB00E0014DB4
:106AB000284638BD0200040038B54D780446032D41
:106AC00009D0212D14D0012D19D1456A1DB11146CF
:106AD0001A46A84738BDE56A1DB120464988A8472F
:106AE00038BD10682946402200F07BFD284638BD9D
:106AF00000F11004146007221A80002038BD0148FC
:106B000038BD00BF0200040008B50346A12018717B
:106B100001294FF0000059719871D871187258729C
:106B20009872D8720BD007D3202910D102211A7382
:106B3000120A99725A730AE00AB101229A71197FF6
:106B40001A1D18680823FFF72FFE002008BD014812
:106B500008BD00BF030001004C2070472DE9F04143
:106B60000C68074614F0030F0D4690468E684B687C
:106B700002D0472B40F28380483B04F14B0223F0C4
:106B8000030322F003022A606B60204600214822A2
:106B900000F027FD3B4B276023643B4B63642B6A6B
:106BA00023626B6A6362AB6AA362EB6AE3622B6B7C
:106BB00023636B6B6363AB6BA363EB6BE363737810
:106BC000042B02D03148BDE8F0817379022BF9D152
:106BD0003379012BF6D8B37823763379012B04D09F
:106BE000EB685A78042AEDD115E033781E443278E8
:106BF000334616445A78052A05D1DA78032AF6D1A5
:106C00009B78237701E0042AF1D1237F002BE7D181
:106C10001F48BDE8F0815A790A2AD3D19A79002A0F
:106C2000D0D19978617619781944187982420FD2B7
:106C30000E78084631444678052E07D1C678022ED4
:106C400004D1807806064CBFA076E0760132ECE7EE
:106C5000A37E002BDCD0E37E002BD9D0696C3846B4
:106C600021B90C49224600F08DFC04E0224600F0D8
:106C700089FC084B6B64C8F80040BDE8F081064809
:106C8000BDE8F081B96A00008D69000008000400C9
:106C900009000400096A00000A00040090F8143298
:106CA00013F01F0305D100F29D12C0F8CC21184645
:106CB00070470148704700BF0100040070477047EB
:106CC00090F8143203F01F03012B06D0022B15D0CD
:106CD000002B37D100F5CF720DE090F89D318BB3CA
:106CE00090F8182290F89B319A422BD20023A0F8FA
:106CF000D43100F5EA72C0F8CC2121E090F81832C6
:106D00001A064BBF4FF48031012103F00F0203F04C
:106D10008F0201FA02F290F89D1109B91B0711D1F7
:106D2000D0F8B4311A420DD0D0F8B8311A420CBFA5
:106D300000230123A0F8D43100F5EA73C0F8CC3168
:106D400000207047004870470100040010B590F81B
:106D5000142212F01F0237D190F81732022B09D0FB
:106D6000032B19D0012B2FD1D0F8A031C0F8CC3192
:106D7000122321E0D0F8AC3190F816128A4205D0E7
:106D80001C780CB15C8823440132F7E71A78DAB139
:106D9000C0F8CC315B880FE0D0F8A43190F81642EF
:106DA000A24204D0197801B10B440132F8E71A78F5
:106DB00052B1C0F8CC311B78B0F8D0219A4288BFCC
:106DC000A0F8D031002010BD004810BD0100040023
:106DD00090F8143203F01F03012B0FD190F89D316E
:106DE00063B190F8183290F89B219A4206D903F5C6
:106DF000E0730344C0F8CC3100207047004870476E
:106E000001000400F8B590F81432044613F01F0393
:106E10000D4602D0022B1BD04AE0B0F81632012BEF
:106E20000ED1036C03B19847B4F89E312DB143F0F5
:106E30000203A4F89E310020F8BD23F00203F8E716
:106E4000022B35D190F81912BDE8F840FFF7A5BC28
:106E500090F818321A0603F08F0105D503F00F02DF
:106E60004FF48036964001E001268E4094F89D2133
:106E7000F2B11B071CD0D4F8B4311E4218D0B4F8BC
:106E80001672AFB935B12046FFF7B4FBD4F8B8316C
:106E90001E430AE0D4F8BC311E42CCD12046FFF795
:106EA000BDFBD4F8B83123EA0606C4F8B861C2E7DE
:106EB0000048F8BD01000400F8B590F814720446CB
:106EC00017F01F0740F0BE8090F81632002B00F03C
:106ED0008480D0F8A851D0F8AC3190F89A21012ADA
:106EE00008BF1D462B78002B00F0A2806B78042B86
:106EF0004ED0052B4ED0022B6CD16A7994F8163205
:106F0000934243D184F89D312B7984F89B3100233F
:106F1000E21801330021082B82F8C011F8D10126B4
:106F200094F899319E4217D20122B240D4F8B4317C
:106F30001A4203D020463146FFF736FB4FF4803229
:106F4000B240D4F8B4311A4204D0204646F0800151
:106F5000FFF72AFB0136E3E74FF00113C4F8B43121
:106F60000023C4F8B831C4F8BC3120460121FFF732
:106F7000D5FAEB7913F0400FB4F89E3114BF43F00B
:106F8000010323F00103A4F89E3123E06B8822E083
:106F9000EF781FE0F7B9AB781A0603F08F0606D535
:106FA00003F00F034FF4803202FA03F301E00123F0
:106FB000B340D4F8B42120461343C4F8B431294671
:106FC000FFF7C6FA20463146FFF7DCFA2046314685
:106FD000FFF7FEFA2B781D4484E780F89D310125E8
:106FE00094F899319D4217D20122AA40D4F8B431C5
:106FF0001A4203D020462946FFF7D6FA4FF48032D2
:10700000AA40D4F8B4311A4204D0204645F0800199
:10701000FFF7CAFA0135E3E700214FF00113C4F886
:10702000B431C4F8B811C4F8BC112046FFF776FAA1
:1070300094F89D0194F81622034B904214BF184611
:107040000020F8BD0048F8BD010004002DE9F74F0D
:1070500090F81432044603F01F03012B40F0918096
:1070600090F89D31002B00F08C80D0F8AC31D0F836
:10707000A85190F89A210026012A08BF1D46434BCB
:10708000B2463746B1462A78002A78D06A78042A70
:107090000AD0052A1CD0022A6ED1697994F89D2164
:1070A000914269D06A8868E095F8029094F81822B5
:1070B000EF7891455DD194F81622974259D104EBAF
:1070C000090393F8C0A183F8C07100231E4653E062
:1070D00094F8182291454FD195F8028018F0800F4E
:1070E00008F08F0B06D008F00F084FF4803202FA38
:1070F00008F803E04FF0010808FA0BF894F816229C
:1071000097421BD1D4F8B421204642EA0802C4F8C1
:10711000B421D4F8B821294622EA0802C4F8B821DB
:107120000193FFF715FA20465946FFF72BFA204640
:107130005946FFF74DFA46EA080618E057451BD1B5
:1071400018EA060F17D1D4F8B4216FEA080802EA4A
:107150000802C4F8B421D4F8B821204602EA080293
:10716000C4F8B82159460193FFF71EFABA46019BAD
:1071700002E0002600E0BA462A78154483E7184664
:1071800000E0024803B0BDE8F08F00BF010004003A
:10719000002100F50572FFF704BBB0F8D03110B53F
:1071A000402B28BF40238021D0F8CC210446FFF794
:1071B000FBFAD4F8CC310344C4F8CC31B4F8D03164
:1071C000181AA4F8D00110BD10B50021D0F8CC21B8
:1071D0000446FFF7A1FAD4F8CC310344C4F8CC310B
:1071E000B4F8D031181AA4F8D00110BD00228021C3
:1071F0001346FFF7D9BA002100F5EA72FFF78CBAFF
:1072000010B580210446FFF7F5F90023A4F8D0312A
:1072100010BDFFFF90F8143213F01F0307D190F850
:10722000162262F07F0280F89C21184670470148C0
:10723000704700BF01000400F8B504460F4605463C
:10724000002694F898319E4213D2D5F858316BB18C
:107250002046D5F878113A469847074B984205D012
:10726000054638B12046FFF7CBFF03E00136043571
:10727000E7E7014D2846F8BD0200040001224FF067
:107280000111A0F89E210022C0F8B41180F89C21C1
:1072900080F89D21C0F8B821C0F8BC210E21FFF76D
:1072A000CBBFFFFF10B50446FFF772FF94F814122E
:1072B0002046C909FFF765F9B4F81A322046A4F848
:1072C000D0310121FFF7B8FF374B98426AD194F8CB
:1072D0001432C3F3411313B1022B50D05EE094F883
:1072E00015320B2B5AD8DFE803F0060F5913591E3D
:1072F000272931333C3EE3682046984700284DD18A
:107300002046FFF74AFF4CE0636A2046002102E076
:10731000636A20460121984700283FD12046FFF7A5
:1073200065FFE36C27E02046FFF774FF002835D1A6
:107330002046FFF75BFF34E02369DDE720460021AC
:10734000FFF758F90023A4F8D0312AE06369D3E7A6
:10735000A3692046984708BB2046FFF747FF636CA8
:1073600009E0E369C8E7236A20469847B0B9204698
:10737000FFF73CFFA36CA3B12046984711E0A36838
:1073800063B120460121984740B9B4F81A32002B66
:10739000CED094F81432DB0903D0B1E72046FFF7D2
:1073A0002FFF002010BD00BF0200040038B590F888
:1073B00014320446DB0923D1B0F8D03113B3FFF700
:1073C00003FFB4F8D031EBB920460221FFF734FFB8
:1073D0000F4B984218D194F81432C3F34113022B87
:1073E0000AD1A36843B1204601219847054618B940
:1073F0002046FFF7FBFE08E02046FFF701FF01E013
:10740000FFF7F9FE002500E00546284638BD00BF1D
:1074100002000400013A10B50446062A40D8DFE80D
:1074200002F0041D21063F3A3C00036817E00421E6
:10743000FFF702FF1B4B984232D194F814122046FA
:10744000C90904D1D4F8CC21B4F8D03103E000212B
:10745000D4F8CC210B46FFF7A2F921E0436820467F
:1074600098471DE090F81432DB0909D00321FFF79B
:10747000E3FE0C4B984213D12046FFF78EFE0FE03F
:1074800090F89C110B060BD501F07F0180F89C1140
:10749000FEF7EAFF04E0002100E08021FFF7BEF8DC
:1074A000002010BD0200040070B515460E464FF4D2
:1074B00007720021044600F094F82A7B254B84F8DB
:1074C0009921A365C4F8D84012B1E365C4F8DC4043
:1074D000214B224A2360224B6360224BE360224B04
:1074E0006362224B2361224B6361224BA361224BD7
:1074F000E361224B2362EB6B002B08BF134623652D
:107500001F4A2B6C002B08BF134663656B6A23640C
:10751000AB6AA3632B69A3626B69E362AB69236304
:107520002B6A6363EB6AE3632B6B63646B6BA3642B
:10753000AB6BE3643368C4F8A0317368C4F8A4315A
:10754000B368C4F8A831F368C4F8AC313369C4F83F
:10755000B03170BD15740000A5720000BD6C000054
:10756000AD730000C16C0000056E00004D6D0000A1
:107570009D6C0000B96E0000D16D00004D700000E0
:10758000BF6C000010B590F89831072B0AD800EBBB
:1075900083040133C4F85811C4F8782180F8983175
:1075A000002010BD004810BD0B00040010B590F87D
:1075B0009941B1EB440F06D800EB81008265C0F819
:1075C000D830002010BD014810BD00BF03000100ED
:1075D00008B500F009F8BDE80840FDF7C9BA00F0A9
:1075E0007FBE00F097BEFFFF10B5174A1749002075
:1075F00000F056F84FF480734FF480620021124877
:1076000000F02EF8124A1349012000F049F84FF417
:1076100080734FF4806200210D4800F021F80E4B7A
:107620001B68022B0EDD0D4A0A49022000F038F8D3
:10763000BDE810404FF480734FF48062002107488A
:1076400000F00EB810BD00BF54040010A684000066
:1076500090040010A8840000AC840000CC0400104A
:1076600070B5C468A50708D0B2F5007F11D0B2F597
:10767000806F04D0B2F5807F0BD0012008E0012399
:1076800000F12401144301610160C361C460002062
:1076900070BD024D5E1EAE42F4D9EEE7FEFFFF0064
:1076A00070B50D4606461046144600F02DF82B78AE
:1076B000722B17D0772B18D0612B23D1082348F2D7
:1076C000020215F8011F2B2912D0622915D01B07C1
:1076D000E260666104D502220021204600F062F8D3
:1076E000204670BD00230122EBE704230222E8E7D5
:1076F00042F0030243F00203E3E742F0040243F0E6
:107700000103DEE70024EBE7F0B5C46889B0A10708
:10771000054622D0220718D4D0E9046700F020F8EB
:10772000384600F010FE230502D5304600F08EF9F1
:10773000A40DA40514F1A54F07D12022296A68469B
:1077400000F010FE684600F0D1F83C2200212846E7
:10775000FFF747FF002009B0F0BD4FF0FF30FAE718
:10776000F7B5044698B103B0BDE8F04000F0EEB8BC
:1077700007FB046000F0EAF8002818BF4FF0FF355F
:107780000134019BA342F3DC284603B0F0BD034B58
:1077900005461B683C270193014EF2E7AC840000CC
:1077A000540400102DE9F843C6683D4B04463340AD
:1077B0000D4690461BB902273846BDE8F883D0F83D
:1077C0001490484600F0C5FD07460028F3D1B8F1F3
:1077D000010F2CD0B8F1020F2ED0B8F1000FEAD172
:1077E000002DE8DBB00404D52368E26A9A4238BF72
:1077F000E362A169A9420EDC2368E26A934238BFC2
:10780000134622695818801AA84204DB206B01EB4A
:10781000000CAC4534DC0023C4E9013346F02006FB
:10782000A56226F4032626F04006E660C4E720465B
:1078300000F038F80544D3E7484600F087FDB0F182
:10784000000CE26804DA42F08002E2600127B3E74C
:10785000E36A1846A3691946236883422CBFC918F6
:1078600009180B4621699206A3EB010303D5A26A0E
:107870009342B8BF13466345ACBFED186544AFE70C
:107880006D1AB10744BF281AA060F10744BF9B1AC4
:10789000EB1A154448BF6360256026F02006C0E758
:1078A00003001000C3689A0705D121220E4B4FF048
:1078B000FF301A60704703F020021B030AD512B193
:1078C000806A0138704703688269006913441B1A93
:1078D000581E70470AB1806A704703688269006960
:1078E0001344181A704700BF5004001010B5044626
:1078F00000F006F801462046BDE8104000F02CBD1F
:1079000010B5421C8307044616D1234654F8041BC5
:10791000A1F1013020EA010010F0803FF5D011F014
:10792000FF0F11D011F47F4F0CD011F47F0F14BF53
:1079300023460333981A04E010F8013B002BE1D1F1
:10794000801A10BD0233F5E70133F3E7C36870B561
:1079500013F00306044611D09B0611D5856A00F08A
:107960008DF8E368204623F44053E36000F00EF8FE
:107970000022064629462046FFF714FF304670BD18
:10798000836905681D440369ED1AEAE738B50446C2
:1079900005690168C36AC06820F40022E26000F053
:1079A0008202022A02D04FF0FF3038BD10F480303E
:1079B000FBD0994238BF19468D4208D10020E368B8
:1079C000E56223F480332560A060E360EDE72246A2
:1079D000491B284600F004F80028EFD0E3E7FFFF3A
:1079E0002DE9F041D5688046EB020E4614465769F2
:1079F00005D5384600F0AAFC45F01005A061124BF1
:107A00002B408BB1A169384600F0A9FC002806DAAA
:107A1000E3684FF0FF3043F08003E36011E025F4AA
:107A2000003525F01005E56032464146384600F045
:107A30009CFC20F00043F61AA3691E44A6610028AE
:107A4000E6D1BDE8F08100BF10000200A8B14FF000
:107A5000805340F80C3C50F8042C72B11368B3F119
:107A6000805F0AD150F8083C516803330B4440F85A
:107A7000083C936840F8043CEDE77047C36810B5D4
:107A800023F02003C3608269836A04469A420ED0C1
:107A9000FFF77CFFE36823F4405323F0100343F027
:107AA0001003E360A36AA3612369E3622360E368D0
:107AB00023F4804323F04003E36010BD2DE9F04739
:107AC00081EA0304C1F30A5640F2FF7704F0004450
:107AD00036B1BE4204D0C3F30A550DB1BD4207D141
:107AE000490011F5001F58D35BD00020344946E00F
:107AF000C1F313014FEAC22841F480113544A1FBC0
:107B000008674FEA525CB6463A46A8FB00674FF05A
:107B10000009B8464CEAC32343F0004C00234FF061
:107B2000000AE0FB0C89ECFB012318EB0E0149EB8A
:107B30000A0A12EB0A0843F10009B9F5801F41EA6D
:107B400096011ED218EB080649EB0900814646EA69
:107B5000D178A5F580654900C80F18EB000249F1FE
:107B60000003B1F1004F40F2FD71164608BF22F04C
:107B700001068D4208D830461C4304EB0551BDE890
:107B8000F087A5F2FF35E7E7002D03DB44F0FF4463
:107B900044F4E00400202146F1E75A0012F5001FEA
:107BA000F8D3084A5B0093429FD811424FF000007F
:107BB0009CD013429AD044F0FF4141F4E001DEE74B
:107BC0000000F87F0000E0FF2DE9F043C1F30A5503
:107BD00040F2FF7C81EA030635B1654504D0C3F36A
:107BE0000A540CB1644506D1454A480090425BD91D
:107BF0000020444956E0A5EB040C440D44EAC121A1
:107C000041F00045510D41EAC32141F000494D4585
:107C10004FEAC0244FEAC22808BF444521BF630889
:107C200043EAC5736A081C4628BF15464FF0000397
:107C30004FF035024FEA580034BF0CF2FD3C0CF215
:107C4000FE3C40EAC9704FEA59018D4208BF8442A8
:107C50004FEA430304D3241A65EB010543F0010303
:107C600024196D41212A08BF1F46013AEDD18D42EA
:107C700008BF844202D3013308BF013740F2FD71CF
:107C80008C4506F0004204D802EB0C52D11918467C
:107C900008E0BCF1000FA4BF42F0FF4242F4E00252
:107CA00000201146BDE8F0835C0014F5001F9FD84A
:107CB000194312EA410301D11249E8E710EA02052B
:107CC00006F0004302D119462846EBE7224005D1D1
:107CD00043F0FF4141F4E0011046E3E714F5001FD3
:107CE00005D043F0FF41002041F4E001DAE710F550
:107CF000001F4FF000003FF47CAF1946D2E700BFF1
:107D00000000E0FF0000F87F944691EA0302F0B41F
:107D100005460E4606D503F100452B46F0BC6246EB
:107D200000F0C6B8994203D3604508D8994206D1FD
:107D300002F10042564053402A466546944640F2BE
:107D4000FF71370D27F40062180D8A42A7EB00047B
:107D500000F0A080944200F09980C6F31302C3F3B0
:107D600013031F2C42F4801143F480134FD823FADD
:107D700004F2891A00F12002D21B93402CFA04F479
:107D80001C432C1B38BF01F1FF311CFA02F32546BE
:107D900003D05B42651E04B9013911F4C01F54D1F0
:107DA000EA0FDB0F42EA410243EA450352EA0304C9
:107DB0006DD0BC1E510B24D0510C01BF190F41EAEC
:107DC00002121B01043CD10C01BF990F41EA82024F
:107DD0009B00023C110D02BFD90F41EA420204F19F
:107DE000FF344FEAD67108BF5B00B1EBD42F4FF0E0
:107DF000000006BF184602EB045106F00041F0BC3B
:107E00007047190E41EA02221B02083CD2E7352CCA
:107E10001BD8203C23FA04F2AA1AC4F1200003FA6A
:107E200000F338BF01F1FF312CFA04F45FEA0C6073
:107E3000154643EA040306D043F0FF035B42551E98
:107E40001AB9013901E0002BF8D1CA0209D4013F67
:107E50007A050FD0EA0F42EA4101DA0F42EA4505FE
:107E60005B00002B21F480124FEA075405DB111947
:107E70002846C4E739051046C1E7013508BF01327D
:107E8000B3F1004F08BF25F00105F0E75CB92146CA
:107E90002046B4E733034FF0000001D00349AEE7BA
:107EA0000CB90249F4E73146E2E700BF0000F87F71
:107EB00091EA030FF0B405460E4605D503F10045DF
:107EC0002B46F0BCFFF720BF994238BF1E4640F258
:107ED000FF7C3EBF0B4615460246300D20F400677E
:107EE000190D6745A0EB01045CD0BC4255D0C6F328
:107EF0001307C3F313031F2C47F4801743F48013B5
:107F000027D82031091A23FA04FC22FA04F48B4002
:107F10002343ED18674428BF013702FA01F3BA0280
:107F20002BD5013508BF01370BB925F00205360DF9
:107F3000360506EB5706730013F5001F2BBF421CD6
:107F400031460020FF0734BF47EA55001105F0BC59
:107F50007047352CE3D8203C23FA04F16D18C4F1A6
:107F6000200103FA01F322FA04F428BF0137234366
:107F7000120618BF43F0FF03D1E7002B00F1FF32D8
:107F800007DA013508BF0137B3F1004F08BF25F00C
:107F9000010507EB02512846D9E74CB906F000412C
:107FA0002046D4E733034FF0000001D00149CEE76B
:107FB0003146F0E70000F87F21F0004230B502F1D1
:107FC000474505F57005B5F17E6F01F000440FD20D
:107FD00002F14843420FC10042EAC30202EBD173EF
:107FE000B1F1004F08BF23F001031C43204630BD10
:107FF000002DFBDB490011F5001F94BF44F0FF4446
:10800000004CF3E70000C07FCB0243EA505040F23F
:108010001E43A3EB115340F00040FF2B20FA03F066
:1080200011D913F4E06F01D14042704711F0804044
:1080300009D04B0013F5001F04D86FF0004000EB8F
:10804000D17070470020704720B9034602461046A1
:1080500019467047030C0CBF000401F18071030E38
:108060000CBF000201F50001030F0CBF000101F578
:108070008001830F0CBF800001F500110028ACBF08
:10808000400001F5801101EBE0234205DFE700F03D
:108090000041002801F18041B8BF4042FFF7D4BF42
:1080A00030B540EA43054C001543254309D09942B9
:1080B00009D1904207D114F5001F8CBF0020012088
:1080C00030BD0120FCE70020FAE730B5054651EA53
:1080D00003000BD4580010F5001F1DD8994219D386
:1080E0001AD195422CBF0020012030BD480010F568
:1080F000001F11D85C0014F5001F0DD82C43144349
:108100002043F2D0994205D806D1954294BF002071
:108110000120EAE70120E8E70020E6E730B551EA70
:10812000030405464FEA41000AD410F5001F1CD88D
:10813000994218D819D1954294BF0020012030BD32
:1081400010F5001F11D85C0014F5001F0DD82C434A
:1081500014432043F3D0994205D306D195422CBF56
:1081600000200120EBE70120E9E70020E7E730B538
:1081700051EA03040BD45C0014F5001F1CD899428B
:108180001CD319D190428CBF0020012030BD4D007E
:1081900015F5001F10D85C0014F5001F0CD899428B
:1081A0000CD801D1904209D22043104350EA050374
:1081B0000CBF01200020E9E70020E7E70120E5E708
:1081C00030B551EA03044FEA41050AD415F5001F02
:1081D0001ED899421ED81BD1904234BF00200120E6
:1081E00030BD15F5001F13D85C0014F5001F0FD823
:1081F00099420FD304D190428CBF00200120EFE7B9
:108200002043104350EA05030CBF01200020E7E79C
:108210000020E5E70120E3E7C20D010241F0004143
:10822000C2F19E039D2A10B5044621FA03F003D93A
:10823000D2B29D2A01D8404210BDFF2A02D1B1F12D
:10824000004FF9D16FF0004303EBD470F4E7FFFF68
:10825000C31013F07F610AD0B1F17F6F4FEA407213
:1082600043F0E04308D003F148411046704703F063
:10827000004300201946704752EA0332014A18BFF2
:108280001346F6E70000F87F884203D00143B1F1BE
:10829000004F06D14000B0F17F4F8CBF002001207D
:1082A00070470020704750EA01034FEA400207D4AC
:1082B000B2F17F4F12D8884294BF0020012070474E
:1082C000B2F17F4F0AD84A00B2F17F4F06D88842F8
:1082D00004D213F1004018BF0120704700207047FE
:1082E00040EA0103DB0703460CD40346043A22BFED
:1082F00051F804CB43F804CBB2F10402F7D20432B4
:1083000008BF7047013A24BF11F801CB03F801CB35
:10831000F8D87047034613F0030F0ED101F0FF01A8
:1083200041EA012141EA0141043A24BF43F8041B18
:10833000B2F10402F9D202F10402013A24BF03F8B7
:10834000011BFAE770474FF0FF3070474FF0FF30E6
:1083500070474FF0FF3070474FF0FF3070474FF0DD
:10836000FF3070474FF0FF30704710467047FFFFF7
:1083700000000000000000000000000000000000FD
:1083800000C001000000000000C01200000000005A
:1083900000C023000000000000C025000000000015
:1083A00000C03600000000000000000000C04800CF
:1083B00000C04900D48300003084000000000000A9
:1083C00000000000000000005084000000000000D9
:1083D00001112202F163000099640000F9630000BA
:1083E000ED670000156400009967000065640000F7
:1083F000696400001D650000516500008365000090
:1084000085650000A9650000D1650000F5650000E4
:108410001D6600009B670000196700009F67000051
:10842000A3670000A96700004564000041660000E2
:1084300085750000AD750000917100009B71000012
:10844000C9710000ED710000F771000001720000B9
:10845000596B00005D6B0000096B00000403090408
:1084600008034E00580050001403560043004F000C
:108470004D00200050006F00720074000E034E008B
:10848000580050002D00370037000A035600430003
:108490004F004D0012010002EF020140C91FDE80B3
:1084A00000010102030172007700FFFF08000000D5
:1084B000C0000B0605000002010000000000FFFFE5
:1084C000C00003000000FFFFC0000409000000FF1F
:1084D000C000080D05000002010000FFC0000815E3
:1084E00000000000000000FFFFFFFFFF09FFFE90FB
:1084F00000EE0000D8FE000000EC000000EB0000E1
:10850000000000FFFFFF000000FFFFFF0800090060
:108510000A000C000F0001FF90D00300010113FFBF
:108520000000803F7593883F8716893F23DB893F92
:10853000BE9F8A3FE3A58B3FCDCC8C3F3F358E3F1E
:108540000000903F2506913FD34D923F46B6933FA2
:108550004260953FC74B973F9A99993F5A649B3F1A
:108560007F6A9C3F68919D3F0000A03F0E2DA23F77
:10857000AAF1A23FA69BA43F6666A63F8B6CA73FCD
:10858000BE9FAA3F2DB2AD3F8D97AE3F0000B03FDA
:10859000AE47B13F3333B33F4260B53F79E9B63FB1
:1085A000FED4B83F713DBA3FD122BB3FA8C6BB3F06
:1085B0000000C03F5839C43F2FDDC43F8FC2C53FC4
:1085C000022BC73F8716C93FBE9FCA3FCDCCCC3FC9
:1085D00052B8CE3F0000D03F7368D13FD34DD23F59
:1085E0004260D53F7593D83F9A99D93F5A64DB3F93
:1085F000560EDD3FF2D2DD3F0000E03F986EE23FD5
:108600008195E33FA69BE43F6666E63F39B4E83FC9
:10861000BE9FEA3FBA49EC3F2DB2ED3FDBF9EE3F9A
:108620000000F03FC1CAF13F3333F33F1D5AF43F1E
:108630004260F53FDD24F63F79E9F63F8B6CF73F6A
:10864000000000000000803F0000803F0000803FED
:108650000000803F0000803F0000803F0000803F1E
:108660000000803F000000400000803F000000400C
:108670000000803F000000400000803F00004040BC
:1086800000000040000040400000803F00008040AB
:1086900000004040000000400000404000008040DA
:1086A0000000803F0000A0400000804000004040EB
:1086B0000000A040000000400000A040000040403A
:1086C000000080400000A0400000C0400000E040EA
:1086D0000000803F000000410000E0400000C0407A
:1086E0000000A040000080400000E040000040404A
:1086F000000000410000A0400000E04000001041E8
:1087000000000040000010410000E0400000A040D8
:1087100000000041000030410000404000002041C6
:108720000000E040000030410000804000001041A7
:108730000000A040000030410000C0400000504157
:108740000000E04000000041000010410000204116
:1087500000003041000040410000504100006041F5
:108760000000803F00007041000060410000504167
:108770000000404100003041000020410000104155
:1087800000000041000070410000E0400000504146
:108790000000C040000030410000A04000006041E7
:1087A0000000104100005041000080400000704176
:1087B000000030410000E040000020410000504136
:1087C00000004040000060410000304100000041D6
:1087D000000050410000A040000040410000E04087
:1087E0000000104100003041000050410000704185
:1087F0000000004000007041000050410000304186
:10880000000010410000E040000040410000A04096
:108810000000504100000041000030410000604174
:108820000000404000005041000020410000E040B6
:1088300000003041000070410000804000005041C5
:1088400000001041000060410000A04000003041E5
:108850000000C040000050410000E04000007041B6
:1088600000000041000010410000204100003041A4
:108870000000404100005041000060410000704194
:1088800000E1F505F11FFF1FB483000009024B0052
:10889000020100C0FA080B000202020004090400F1
:1088A0000001020200040524001001052401010159
:1088B00004240202052406000107058203100002B9
:1088C00009040100020A000004070501024000003B
:0888D0000705810240000000D1
:00000001FF
